:200000000C945C000C946E000C946E000C946E000C946E000C946E000C946E000C946E0082
:200020000C946E000C946E000C946E000C946E000C946E000C946E000C946E000C946E0050
:200040000C9412010C946E000C946E000C946E000C946E000C946E000C946E000C946E008B
:200060000C946E000C946E0000000000240027002A0000000000250028002B000404040467
:200080000404040402020202020203030303030301020408102040800102040810200102F1
:2000A00004081020000000080002010000030407000000000000000011241FBECFEFD8E063
:2000C000DEBFCDBF21E0A0E0B1E001C01D92A930B207E1F70E945C010C94CB010C94000000
:2000E000ECEAF0E02491E8E9F0E09491E4E8F0E0E491EE23C9F0222339F0233001F1A8F4B5
:20010000213019F1223029F1F0E0EE0FFF1FEE58FF4FA591B4912FB7F894EC91811126C0B7
:2001200090959E239C932FBF08952730A9F02830C9F0243049F7209180002F7D03C0209139
:2001400080002F7720938000DFCF24B52F7724BDDBCF24B52F7DFBCF2091B0002F77209385
:20016000B000D2CF2091B0002F7DF9CF9E2BDACF3FB7F8948091050190910601A0910701ED
:20018000B091080126B5A89B05C02F3F19F00196A11DB11D3FBFBA2FA92F982F8827BC01A6
:2001A000CD01620F711D811D911D42E0660F771F881F991F4A95D1F708958F929F92AF92C3
:2001C000BF92CF92DF92EF92FF920E94B8004B015C0184E6C82ED12CE12CF12C0E94B80006
:2001E000681979098A099B09683E734081059105A8F321E0C21AD108E108F10888EE880E11
:2002000083E0981EA11CB11CC114D104E104F10429F7FF90EF90DF90CF90BF90AF909F90FE
:200220008F9008951F920F920FB60F9211242F933F938F939F93AF93BF9380910101909165
:200240000201A0910301B09104013091000123E0230F2D3758F50196A11DB11D20930001A1
:200260008093010190930201A0930301B09304018091050190910601A0910701B091080102
:200280000196A11DB11D8093050190930601A0930701B0930801BF91AF919F918F913F91C1
:2002A0002F910F900FBE0F901F90189526E8230F0296A11DB11DD2CF789484B5826084BDAA
:2002C00084B5816084BD85B5826085BD85B5816085BD80916E00816080936E001092810004
:2002E0008091810082608093810080918100816080938100809180008160809380008091D9
:20030000B10084608093B1008091B00081608093B00080917A00846080937A0080917A0098
:20032000826080937A0080917A00816080937A0080917A00806880937A001092C100E8E921
:20034000F0E02491E4E8F0E08491882399F090E0880F991FFC01E859FF4FA591B491FC0170
:20036000EE58FF4F859194918FB7F894EC91E22BEC938FBFC0E0D0E081E00E9470000E9420
:20038000DD0080E00E9470000E94DD002097A1F30E940000F1CFF894FFCFFFFFFFFFFFFF8E
:2003A000FFFFFFFFFFFFFFFFFFFFFFFFFFFFFFFFFFFFFFFFFFFFFFFFFFFFFFFFFFFFFFFF5D
:2003C000FFFFFFFFFFFFFFFFFFFFFFFFFFFFFFFFFFFFFFFFFFFFFFFFFFFFFFFFFFFFFFFF3D
:2003E000FFFFFFFFFFFFFFFFFFFFFFFFFFFFFFFFFFFFFFFFFFFFFFFFFFFFFFFFFFFFFFFF1D
:20040000382F10C8ACBA2F102834FA00007B000008142A142222142A14085500550055AA86
:2004200055AA55AAFF55FF55FF000000FF00101010FF00141414FF001010FF00FF1010F080
:2004400010F0141414FC001414F700FF0000FF00FF1414F404FC141417101F10101F101F50
:200460001414141F00101010F0000000001F101010101F10101010F010000000FF10101014
:20048000101010101010FF10000000FF140000FF00FF00001F10170000FC04F41414171053
:2004A000171414F404F40000FF00F714141414141414F700F7141414171410101F101F14B8
:2004C0001414F4141010F010F000001F101F0000001F14000000FC140000F010F01010FF3C
:2004E00010FF141414FF141010101F00000000F010FFFFFFFFFFF0F0F0F0F0FFFFFF0000A7
:20050000000000FFFF0F0F0F0F0F3844443844FC4A4A4A347E02020606027E027E02635500
:200520004941633844443C04407E201E2006027E020299A5E7A5991C2A492A1C4C720172BF
:200540004C304A4D4D303048784830BC625A463D3E494949007E0101017E2A2A2A2A2A447A
:20056000445F444440514A444040444A51400000FF0103E080FF000008086B6B08361236C4
:200580002436060F090F06000018180000001010003040FF0101001F01011E00191D17126F
:2005A000003C3C3C3C00000000000000000800020100000304070000000000000000000032
:2005C0000000250028002B0000000000240027002A00040404040404040402020202020202
:2005E000030303030303010204081020408001020408102001020408102011007F9629001D
:2006000001007F9628003A0155F603090103B00140B40100C00123C10110C5022B2BC701C5
:20062000C0360188B102001BB70107C0021010C10141C50400228040360168B00100B1021B
:20064000B011B40102B60302023BB701C63A0155F704A9512C82C0020D0DC1024300C201D4
:2006600000C50400480048B40100B60302023BE00F0F211C0B0E08499838091103141000BE
:20068000E10F0F2F2B0C0E06477637071104231E00B00100B30402000000B40100D0030797
:2006A0004218D103000710D2020102D3020102D4020102C005103B000211C103101088C519
:2006C0000103C60102C80C003236450616377577540C00CC0100F603010100CF03008130E2
:2006E000ED0464031281E803851078CB05392C003402F70120EA020000B00100B102001B29
:20070000B40100C00121C10111C5023F3CC701B5360148F20100260101E00F0F26240B0EB5
:200720000954A8460C17090F0700E10F00191B0410072A473903060630380F360100B001D5
:2007400000C10410100202C006003500000102C50104D2020104CA0100EA0180B00100B276
:20076000050C0C003333B70135BB012BC00104C20201FFC30111C40120C6010FD002A4A1F2
:20078000E00ED000050E150D3743470915121619E10ED000050D0C062D44400E1C18161941
:2007A0003A01557F0AB00103E2013FC00122E20100B00100C0010AB0010000000000000057
:2007C00000000000000000000000FFFF0F0000040062080008080003000C01030B5A020311
:2007E0000609030317100403002305030017060309630703090C08030C1009033222100049
:20080000160011000101120000001300010000013003010137020301000D80020061020123
:20082000B0C1FFFF3200010000010200000103003010090001000C000000900000800F009A
:200840000000100200001102EF001202000013028F01000500000105000002055F00010455
:20086000010004040000FFFF320007000001FFFF3200000200000102000000000000000002
:2008800000000000000000000100A4000100FFFF0A00600000270800080830001402310094
:2008A0001537320004063300160E340011223500001536000785370007143800031439000C
:2008C0002000900015001000100411003702290046002A0046000700000012008901130050
:2008E0000011FFFF96001200B901010000010200000203003010090001000A0000000D001D
:2009000000000E003000610001006A000000800000008100000082005F00920000019300C5
:200920000107FFFF500007000001E500F078010000010200000203003010040000000500BA
:20094000000008000702090000000A0000000C0000000D0000000F0000001000000011002A
:200960000700120000001300000007000100FFFFC8001000901611002702FFFF320012004B
:200980000D00FFFF32001300001229000A002B000D00FFFF320020000000210000003000E9
:2009A0000000310004043200030035000504360008083700070438000303390007073C0042
:2009C00004053D00080860000027610001006A000000800000008100000082000000830068
:2009E00000008400000085000000900010009200000007003301E50000800000010001001A
:200A0000000102000007030030100400000008000202090000000A0000000C0000000D004D
:200A200000000F00000010000000110007001200000013000000FFFF32001000B017110042
:200A40000700FFFF0A0012003A01FFFF0A001300001A29000C00FFFF0A0030000000310067
:200A600005053200040035000600360007073700050138000200390007073C0004073D0075
:200A80000708600000A7610001006A000000210000002000000080000000810000008200B0
:200AA0000000830000008400000085000000900010009200000093000300950010019700A5
:200AC00000009800000007007301FFFF3200FF000100F300080000000100010000010200D3
:200AE000000703003010080002030900000010000000110007001200000013000000FFFF4B
:200B000032001000B014FFFF0A0011000700FFFF0A0012008E001300000C29001500FFFFAC
:200B20000A00300000003100070132000000350003023600020437000000380007023900E9
:200B400000003C0003023D000304600000A7610001009000290007003301FFFF320015006E
:200B600030009A00100011002000100028341200020013003810FFFF280012001200FFFF47
:200B800028001000203413004530FFFF4600300000003100020432000703330004033400EC
:200BA0000400350001043600070737000503380010063900100601000001020000030300CD
:200BC0003010080008080A000800600000276100010090003E019200000193000001A0002C
:200BE0000030A3001000070001000700210007002300070033000700330111001A00120006
:200C0000213113006C001400494210000008FFFF0A0011001A01FFFF0A0011001A03FFFFE4
:200C20000A0011001A07FFFF0A0011001A0FFFFF0A0011003A0FFFFF1E000100280102008C
:200C400000010300301007001210080003030B0000110C0000000F00011815002000500044
:200C6000010151000306520008045300000054000506550006045600030357000303580098
:200C800010005900001007001200FFFF28000700130007001700B22311241FBECFEFD8E007
:200CA000DEBFCDBF11E0A0E0B1E0EAE8F8E502C005900D92AA3CB107D9F722E0AAECB1E0CD
:200CC00001C01D92A138B207E1F716E0CCE4D6E004C02197FE010E94382CCB34D107C9F7C6
:200CE0000E94D9230C94432C0C9400004398429825B12C7F392F3370232B25B92BB12370CB
:200D00009C7F922B9BB94198419A95B19C7F282F2370922B95B99BB193708C7F892B8BB94B
:200D20004198419A429A85B18C7F972F9370892B85B98BB183707C7F782B7BB94198419A72
:200D400085B18C7F962F9370892B85B98BB183706C7F682B6BB94198419A439A08950895FC
:200D6000E5E4F2E027A930AD98E0699FB0011124607E777050E093E0559547959A95E1F790
:200D8000462B572B90E0982F88278827987F842B952B96AB85AB918B808B338B228B0895A5
:200DA000AF92BF92CF92DF92EF92FF920F931F93CF93DF936C017B018B01040F151FEB01ED
:200DC0005E01AE18BF08C017D10759F06991D601ED91FC910190F081E02DC6010995892B2B
:200DE00079F7C501DF91CF911F910F91FF90EF90DF90CF90BF90AF90089590E0FC01E655EE
:200E0000FA4F2491FC01EA51FA4F3491FC01EE52FA4FE491EE23C9F0222339F0233001F116
:200E2000A8F4213019F1223029F1F0E0EE0FFF1FE254FA4FA591B4918FB7F894EC916111A9
:200E400026C030953E233C938FBF08952730A9F02830C9F0243049F7809180008F7D03C0D7
:200E6000809180008F7780938000DFCF84B58F7784BDDBCF84B58F7DFBCF8091B0008F779A
:200E80008093B000D2CF8091B0008F7DF9CF3E2BDACF3FB7F8948091400290914102A091DD
:200EA0004202B091430226B5A89B05C02F3F19F00196A11DB11D3FBFBA2FA92F982F8827B6
:200EC000BC01CD01620F711D811D911D42E0660F771F881F991F4A95D1F708958F929F921A
:200EE000AF92BF92CF92DF92EF92FF926B017C010E9449074B015C01C114D104E104F10474
:200F0000B9F00E944907681979098A099B09683E73408105910580F321E0C21AD108E10875
:200F2000F10888EE880E83E0981EA11CB11CE4CFFF90EF90DF90CF90BF90AF909F908F909E
:200F4000089581E08093440284B1836084B98AB18C6F8AB9389A399A3A9A3B9A3C9A439A6B
:200F6000409A419A449A62E370E080E090E00E946E07449864E670E080E090E00E946E0705
:200F8000449A64E670E080E090E00E946E0770E060E080EB90E00C947606CF93DF93C82FA0
:200FA000D62F80914402811102C00E94A1074398429885B18C7F85B98BB183708BB94198B7
:200FC000419A95B19C7F8C2F8370982B95B98BB18370CC7F8C2B8BB94198419A84B18C7FAD
:200FE00084B98AB183708AB9429A61E070E080E090E00E946E07409A40984098409893B149
:2010000039B1409A409A40984098409883B129B1409AD15080F7409A439A44B1436044B9DE
:201020004AB14C6F4AB993703C7F932B83702C7F822BDF91CF9108950F931F93CF93DF939B
:201040008C0160E00E94CD07EC0161E0C8010E94CD078C01BE0190E080E0CB0177276627CD
:2010600030E020E0602B712B822B932BDF91CF911F910F910895FF920F931F93CF93DF9358
:201080008C0160E00E94CD07EC0161E0C8010E94CD07F82E62E0C8010E94CD07AE0170E0FA
:2010A00060E0742F66275527442700E030E020E0402B5F29622B732B292F30E0C901B0E009
:2010C000A0E08A019B01082B192B2A2B3B2BC901B801DF91CF911F910F91FF9008950F93C6
:2010E0001F93CF93DF93EC018B01FE0125913491FE0132962496659174912F3F320771F4EF
:2011000090E080E00E946E07045011091016110664F3DF91CF911F910F9108954398429874
:2011200085B18C7F932F9370892B85B98BB18370932F9C7F892B8BB94198419A85B18C7FBE
:20114000922F9370892B85B98BB183702C7F282B2BB94198419A429A85B18C7F972F93702E
:20116000892B85B98BB18370972F9C7F892B8BB94198419A85B18C7F962F9370892B85B9C6
:201180008BB183706C7F682B6BB94198419A439ABBCF4398429895B19C7F95B99BB19370B0
:2011A0009BB94198419A95B19C7F282F2370922B95B99BB193708C7F892B8BB94198419ACB
:2011C000FA01615080F02191429A95B19C7F822F8370982B95B98BB183702C7F822B8BB984
:2011E0004198419AEECF439A0895DF92EF92FF920F931F93CF93DF93CDB7DEB768970FB67C
:20120000F894DEBF0FBECDBF7C018B01F70184913196D490F2E0EF0EF11C8F3779F0DE0121
:20122000119630E020E0AD012D1528F5F701E20FF31FE491ED932F5F3F4FF6CF6D2D70E02F
:2012400090E080E00E946E07D12CED2DF0E032960E1B1F0B10161106CCF268960FB6F8945B
:20126000DEBF0FBECDBFDF91CF911F910F91FF90EF90DF900895ED0CF11C6D2D90E00E948C
:20128000C908E3CFFC01262F358D868D82958170982F9627692F70E072A361A330FF0CC01C
:2012A000821307C080E290E050E040E060E00C94C90881E290E0F8CF878D90A1833927E756
:2012C000920741F058F4843521E0920789F08032944559F4626081E094E011C0863223E928
:2012E0009207C1F38930954BA9F381E690E007C0660F771F660F771F636187E090E00C947D
:2013000076068F929F92AF92BF92CF92DF92EF92FF920F931F93CF93DF9300D000D0CDB73D
:20132000DEB77C014B015A016901FC01878D90A18732F3E99F0709F041C0F701868982305A
:20134000A1F5F0E2AF0EB11C005E1F4FF70187A190A5258D20FF49C099828A82DB82CC82CE
:20136000AE014F5F5F4F64E090E00E94C908F70181A5B982AA821B830C83AE014F5F5F4F7E
:2013800064E090E00E94C9080F900F900F900F90DF91CF911F910F91FF90EF90DF90CF90AE
:2013A000BF90AF909F908F900895833079F620E2820E911C80E2C80ED11CC8CF8632954109
:2013C00029F6F701868980FFC1CFC801841B950B19F40F5F1F4FBACF6217730709F0B6CFED
:2013E0006B01C80ED91E8A01B1CFB4010E947606B501F70181A592A50E947606F701858DA3
:2014000085FF08C0868980FF1EC0102F0027A02AB12A8501B401F70185A596A50E94760653
:20142000B501F70181A992A90E947606B601F70187A590A90E947606B801F70183A994A92F
:201440000E947606A1CFDC2CCC248C289D286401E1CFAF92BF92CF92DF92EF92FF920F9360
:201460001F93CF93DF93EC0137FF05C0620F731F319521953109260F371F77FF02C070E032
:2014800060E088859985281739070CF4C9016C01C61AD70A17FF05C0400F511F1195019594
:2014A0001109040F151F57FF02C050E040E02A853B85021713070CF498015901A41AB50A51
:2014C0008901015011099C0121503109CE010E948109439842983BA58CA525B12C7F982FC6
:2014E0009370292B25B99BB193708C7F982B9BB94198419A95B19C7F832F8370982B95B97B
:201500008BB183703C7F832B8BB94198419ACA14DB042CF09A2D8B2D5601C92ED82E429AB3
:201520009F2D93702F2D2C7FF22E4E2D43708E2D8C7FE82E1C141D04E4F4950185B18C7FAB
:20154000892B85B98BB183708F298BB94198419A85B18C7F842B85B98BB183708E298BB962
:201560004198419A2150310949F721E0C21AD108E1CF439A8D8D80FF08C08F8D98A186321B
:20158000954191F48E8980FF0FC00A851B8501501109288539852150310950E040E070E03B
:2015A00060E0CE010E948109DF91CF911F910F91FF90EF90DF90CF90BF90AF900895EF9248
:2015C000FF920F931F93CF93DF93F901EA01C81BD90B9E012F5F3F4FDF01A61BB70B8D01FA
:2015E0000F5F1F4F37FF04C09E0120953095CA0117FF04C08D0100951095BF01E0907A02E3
:20160000F0907B02AB01BC0185E492E00E94290ADF91CF911F910F91FF90EF900895CF9288
:20162000DF92EF92FF920F931F93CF93DF9300D000D0CDB7DEB78C017A01690177FD3DC063
:2016400057FD3BC0FC018085918568177907ACF5828593854817590784F5878D90A187322E
:20166000934939F4F80186898230A1F5F0E2EF0EF11CF80187A190A5258D20FF30C0798322
:201680006A837B836C83AE014F5F5F4F64E090E00E94C908F80181A5F982EA82FB82EC824D
:2016A000AE014F5F5F4F64E090E00E94C908B601F80183A594A50E9476060F900F900F90EC
:2016C0000F90DF91CF911F910F91FF90EF90DF90CF900895833069F6605E7F4FCACF0E94F9
:2016E0007606B701F80181A592A50E947606DFCFAB0120917A0230917B02BC0185E492E0E5
:201700000C940F0BEF92FF920F931F93CF93DF93CDB7DEB72A970FB6F894DEBF0FBECDBFB4
:201720007C01862F8370F701868B962F917060FFF1C026813781F70131872087992309F436
:20174000ECC024813581F70133872287823009F4E9C0833009F4E8C0813009F4E1C088E4BC
:201760008A87F701258D368D30FF03C08A8580588A8731FF04C08A8590E489278A8733FF97
:2017800004C08A8598E089278A87F701878D90A120FF12C18431F8E69F0709F0C7C09A8536
:2017A000892F88728A871F82892F85958074282F2260892F90E09595879580729927822B59
:2017C00088878BE38987AE01495F5F4F63E086EB90E00E94C9082AE230E0F70130A727A32B
:2017E0008BE290E092A781A74CE250E054A743A736A725A730AB27A792AB81AB94AB83AB40
:20180000AE01465F5F4F61E086E390E00E94C9088A8590E0F70194A383A3F701868980FFDF
:201820001CC0858D968D92FD18C087A190A521A532A530A727A392A781A785A596A521A905
:2018400032A936A725A792AB81AB87A590A923A934A930AB27A794AB83ABF7010285138560
:2018600001501109208531852150310950E040E070E060E0C7010E948109F701668177814C
:20188000878D90A110E000E020E08732F3E99F0769F4F7012689225010E000E0223010F45C
:2018A00000E210E020E230E0201B310BF701458D40FF3CC119820A837B836C831D822E8362
:2018C000AE014F5F5F4F66E083E390E00E94C90819820A83AE014F5F5F4F62E087E390E01F
:2018E0000E94C908F701858D80FF07C050E040E060E083E190E00E94C9082A960FB6F8943D
:20190000DEBF0FBECDBFDF91CF911F910F91FF90EF900895248135810ECF2681378113CF8D
:2019200088E21ECF88E91CCF88EF1ACF833629E1920769F0813844E9940749F08131E5E1AD
:201940009E0729F08138F5E19F0709F044CF2A8527FF02C021602A872A8526FF2EC122607A
:201960002A878138954151F483E18F83AE01495F5F4F61E080EC90E00E94C908F701878DCB
:2019800090A18336F9E19F0721F48A858F738A8722CF813824E9920721F0813845E19407CB
:2019A00019F42A852F722A878131954109F013CF8A858F7E806CEBCF6A85262F062E000C70
:2019C000330B8339F7E79F0761F008F042C08435E1E09E0709F46AC08032F4E59F0709F0CE
:2019E00041C040E052E0F70150A747A341E052E052A741A742E052E054A743A740E152E0FB
:201A000056A745A741E152E050AB47A742E152E052AB41AB43E152E054AB43AB222730782E
:201A20008632F3E99F0729F060E07AE68032944511F460E075E3622B732B80E094E00E94EA
:201A400076066A85F4E06F9FB00111246627717055C0863243E9940721F28930E5EB9E0710
:201A600009F4BFCF80E290E0F70190A787A381E290E092A781A782E290E094A783A780E5DE
:201A800090E096A785A781E590E090AB87A782E590E092AB81AB83E590E094AB83ABB901EF
:201AA00066277078776280E690E0C9CF87E390E0F70196A785A786E390E090AB87A789E381
:201AC00090E092AB81AB88E390E094AB83AB80E290E090A787A381E290E092A781A782E21A
:201AE00090E094A783A7F4E06F9FB001112466277170222732702862622B732B81E090E06A
:201B00000E9476068A85682F70E075956795759567956870772783FD70616063F70174A30C
:201B200063A383E090E00E94760677CE8338F7E79F0721F198F4843541E0940751F1803223
:201B40009445B9F4F70161A172A1626081E094E00E947606B80184E094E02CC08632F3E92C
:201B60009F0781F3893025EB920761F38339974749F3F70161A172A1626003C0F70161A133
:201B800072A181E690E00E947606B8018AE690E011C0600F711F6150710981E390E00E9433
:201BA0007606B80182E390E00E94760670E060E083E390E00E947606A0CE8138954109F083
:201BC000DDCE82E1D2CE2091F101260F3327331F21323105ECF420911502FC0190E080E0D5
:201BE000243069F082E00895A091F1012191AC014F525E4FA40FB52FB11D2C930196861711
:201C000098F38091F101680F6093F10180E0089581E008958FEF9FEF08958FEF9FEF08958D
:201C20008091CA0190E09195819591090895CF93DF93CB01EA01642F0E94E30DCE01DF91F6
:201C4000CF910895CF93DF931F92CDB7DEB7698361E0CE0101960E94E30D81E090E00F9054
:201C6000DF91CF9108950895FC016370668B8481958126813781613039F0633029F09187A1
:201C80008087338722870895318720879387828708952F923F924F925F926F927F928F9287
:201CA0009F92AF92BF92CF92DF92EF92FF920F931F93CF93DF93CDB7DEB76A970FB6F894EA
:201CC000DEBF0FBECDBF9A8F898F7A8369834A01D22E18870F833701BC2CDC0159962D91BE
:201CE0003C915A972115310509F015C118968D919C911997681779070CF0D7C11A968D91E1
:201D00009C91481759070CF0D0C14C2C512CB6E0CB9E600D711D11247C876B8716161706E8
:201D20000CF0C3C1EA2DF0E0FA87E98793E0EE0FFF1F9A95E1F7F88BEF87CF01840F951FA6
:201D4000181619060CF0B1C1A98DBA8D58968C91811104C0BFEABD1508F4D394A98DBA8D8F
:201D6000ED91FC9111970284F385E02DCD010995B5E0DB9EC0011124E981FA81FC83EB8363
:201D8000312C212C9C0126553F4F388F2F8B4A2D50E05E8B4D8BEF89F88DE20DF31D449139
:201DA0009E828D82D12CC12C69817A81620D731D7A8B698B842F90E09C8B8B8BE98DFA8DD0
:201DC000A081B18140FF82C0F1E0BF126FC0AF126DC01C96ED91FC912F813885A4014C0D48
:201DE0005D1D69897A89898D9A8D0995EB89FC89F595E7954E2F5FEFC51AD50A6D817E8124
:201E00008D899E89680F791F7E836D8398E0C916D10481F6AFEF2A1A3A0AEB81FC81E40DE2
:201E2000F51DFC83EB83F5E02F16310409F0B3CF2F81388526153705B9F0A98DBA8DED9151
:201E4000FC91B1E0BB1257C0AB1255C069817A816B5F7F4F0088F189E02D830128E030E086
:201E6000A401898D9A8D0995A98DBA8DED91FC9111970688F789E02DCD016A960FB6F89478
:201E8000DEBF0FBECDBFDF91CF911F910F91FF90EF90DF90CF90BF90AF909F908F907F9065
:201EA0006F905F904F903F902F9009941E96ED91FC91EF80F88409851A8592014D815E8113
:201EC0006B817C81898D9A8D099590CF2F8138852615370509F48ACF31E0B31207C0A31253
:201EE00005C01C96ED91FC91930178CF1E96ED91FC917301E0CF6B857C856419750906842D
:201F0000F785E02D73010F8518899201A401898D9A8D0995A9CFF90134969491329745917C
:201F20005491D91AB7E0DB9E400D511D1124F901259134913C8B2B8BFA0125903490FA0168
:201F40003296749031963491398B329664903196449041E04C1518F04A1508F07FC0662D5B
:201F6000062C000C770B7C836B83842D042C000C990B9E838D83A98DBA8DED91FC911197C2
:201F80000284F385E02DCD010995512CD12CC12CEA2DF0E0FA87E9872B2D30E03C872B87AE
:201FA000A401440D511D47FC5A95588F4F8B69817A81660D711D67FC7A957E876D87798977
:201FC000C71608F051CF2C2D30E04D815E81420F531FA985BA854A9FC0014B9F900D5A9F9C
:201FE000900D1124FC01E80DF91DF88BEF87852D612C4F89588D420F531F5E8B4D8B671413
:2020000008F050C044244394480E877041F4C1010196EB89FC89E20DF31DD4901C01D7FE50
:2020200019C0A98DBA8DED91FC91662D70E0B1E0BB1219C0AB1217C02D853E85620F731F19
:202040000484F585E02D2F8138854D895E89898D9A8D0995DD0C6394842DD1CF1E821D82FC
:202060001C821B8288CF4B815C81640F751FAB85BC856A9FC0016B9F900D7A9F900D112451
:2020800069817A81680F791F0684F785E02DEF80F88409851A859D014F855889898D9A8D91
:2020A0000995D8CF570CC3948ACF6A960FB6F894DEBF0FBECDBFDF91CF911F910F91FF90D2
:2020C000EF90DF90CF90BF90AF909F908F907F906F905F904F903F902F9008958F929F927E
:2020E000AF92CF92EF92FF920F931F93CF93DF93EC01262F898D9A8D009709F051C06A304A
:20210000D1F41D861C868D8948E0849F900111248E859F85820F931F9F878E8781E090E008
:20212000DF91CF911F910F91FF90EF90CF90AF909F908F9008956D3089F3CC88AD888F892E
:202140008823C1F08C859D8536E0C39E800D911D1124488559854817590764F44E855F8590
:202160001D861C8638E0A39EC0011124840F951F9F878E87EA88FB88088919894E855F856A
:202180006C857D85CE010E94490E2C898C859D8546E0249F800D911D11249D878C87BECF7F
:2021A0006A3069F41D861C86FC013896E4912D898E859F85E29F800D911D1124ADCF6D30AC
:2021C00009F4ACCFFC0134963491631708F4A6CF3296E491E61708F4A1CFFC013296859090
:2021E0009490462F431B342F47E0349F800C911C1124F401329634913196E4913323A9F16F
:20220000EE2399F1CC88F4013596E491AD884F89442301F10E2E000CFF0BE30FF11DCE9E76
:20222000A001CF9E500D11246C857D85460F571F68857985641775076CF44E855F851D86A4
:202240001C86FC013896E491AE9E400D511D11245F874E87EA88FB88088919894E855F85C6
:202260006C857D85CE010E94490EF4013496E4912C898C859D85E29F800D911D11248DCF3A
:202280006F927F928F929F92AF92BF92CF92DF92EF92FF920F931F93CF93DF93EC016B01E3
:2022A0005A0139014801E881F9810284F385E02D0995E881F9810288F389E02D87019301A2
:2022C000A501B601CE010995A501480D591D41505109E881F9810288F389E02D9301B60197
:2022E000CE010995E881F9810088F189E02D9401A501B601CE010995C60CD71CB6016150F3
:202300007109E881F9810088F189E02D9401A501CE010995E881F9810688F789E02DCE01DC
:20232000DF91CF911F910F91FF90EF90DF90CF90BF90AF909F908F907F906F9009946F9219
:202340007F928F929F92AF92BF92CF92DF92EF92FF920F931F93CF93DF935C01EB016A01C8
:20236000490138018701DC01ED91FC916217730719F5641675062CF0962D872D3A01C92EAF
:20238000D82E9601261937092F5F3F4F048CF58DE02DA301BE01C5010995DF91CF911F919F
:2023A0000F91FF90EF90DF90CF90BF90AF909F908F907F906F9008954615570591F42617A1
:2023C000370724F0892D4B01C22FD82F9E01281939092F5F3F4F068CF78DE02DA601B401F4
:2023E000DACF0284F385E02D0995D501ED91FC910488F589E02D83019401A601BE01C5014E
:202400000995D501ED91FC910688F789E02DC501DF91CF911F910F91FF90EF90DF90CF9060
:20242000BF90AF909F908F907F906F900994EF92FF920F931F93E0907A02F0907B0289013C
:202440009A01AB01BC0185E492E00E949F111F910F91FF90EF900895EF92FF920F931F93EA
:20246000DC011A960D911C911B9718962D913C911997ED91FC9100A0F1A1E02D7B0150E0F3
:2024800040E070E060E009951F910F91FF90EF9008954F925F926F927F928F929F92AF927C
:2024A000BF92CF92DF92EF92FF920F931F93CF93DF936C012B015A0139014801DC01ED91ED
:2024C000FC910284F385E02D0995E201640C751CD601ED91FC91C615D7055CF40088F189F7
:2024E000E02D87019401A501BE01C60109952196EFCF0688F789E02DC601DF91CF911F9111
:202500000F91FF90EF90DF90CF90BF90AF909F908F907F906F905F904F9009948F929F9298
:20252000AF92BF92CF92DF92EF92FF920F931F93CF93DF93EC015B014A016901E881F9811C
:202540000284F385E02D099595012C0D3D1D21503109E881F9810488F589E02D7801840106
:20256000A401B501CE010995E881F9810688F789E02DCE01DF91CF911F910F91FF90EF9098
:20258000DF90CF90BF90AF909F908F9009948F929F92AF92BF92CF92DF92EF92FF920F938A
:2025A0001F93CF93DF93EC015B014A0169017801E881F9810284F385E02D0995C80CD91CC9
:2025C000860101501109E881F9810488F589E02D9501A401B501CE010995E881F981068840
:2025E000F789E02DCE01DF91CF911F910F91FF90EF90DF90CF90BF90AF909F908F9009940A
:20260000EF92FF920F931F93DC01ED91FC9100A0F1A1E02D09951F910F91FF90EF90089594
:202620000F931F93DC01ED91FC91068CF78DE02D09951F910F9108950F931F93DC01ED9101
:20264000FC91048CF58DE02D09951F910F9108952F923F924F925F926F927F928F929F927B
:20266000AF92BF92CF92DF92EF92FF920F931F93CF93DF93CDB7DEB72C970FB6F894DEBFF2
:202680000FBECDBF3C017C836B835C874B871801270181E090E05C01A41AB50ACA01919525
:2026A00081959109AC01440F551F5A834983C80101969E838D83F12CE12C88248394912C12
:2026C000922F91709F8322702887AB014F5F5F4F5A8749878B859C85E816F9060CF07AC0B8
:2026E000CB84DC84B7FC0CC06C0191E0C91AD10849815A814E5F5F4F5A834983A40EB51EE4
:202700005FEFE51AF50A82E0880E911CA80CB91CCE14DF0464F19F81992399F09601220FF8
:20272000331F4D815E81240F351F82014B815C814C195D09B701660D771D85E492E00E94E0
:202740001C135885552399F09601220F331F8D819E81280F391F82014B815C814C195D099F
:20276000B3016E197F0985E492E00E941C134B855C854C155D0559F15F81552391F09401BE
:2027800022503109220D331D820149855A854E195F096B857C85660D771D85E492E00E949A
:2027A0001C138885882399F0940122503109220D331DB3014B855C85641B750B8201498534
:2027C0005A854E195F0985E492E00E941C13DC86CB8680CF2C960FB6F894DEBF0FBECDBF94
:2027E000DF91CF911F910F91FF90EF90DF90CF90BF90AF909F908F907F906F905F904F9025
:202800003F902F9008952F923F924F925F926F927F928F929F92AF92BF92CF92DF92EF92E0
:20282000FF920F931F93CF93DF9300D000D0CDB7DEB71C012B015A0169014701421753071D
:202840000CF05EC05A8349839A0157FD5DC089819A81959587959A83898329813A813C83F1
:202860002B830217130714F41C830B836B807C80660C771C8B819C81820D931D9A838983C5
:2028800095012619370974018601A201BC0185E492E00E940013C618D70891E0C91AD1084D
:2028A0002B813C81420E531EA20CB31CC501821B930B860121E04B815C81B20101970E9452
:2028C000281322E04B815C81B20189819A810E9428130F900F900F900F90DF91CF911F9161
:2028E0000F91FF90EF90DF90CF90BF90AF909F908F907F906F905F904F903F902F90089579
:202900003A83298337FFA3CF2F5F3F4F3A8329839ECFDC01ED91FC910084F185E02D099428
:202920002F923F924F925F926F927F928F929F92AF92BF92CF92DF92EF92FF920F931F9305
:20294000CF93DF9300D000D0CDB7DEB76C015B015C834B8381E090E04C01841A950A2A01EE
:20296000519441945108440C551CF12CE12C66246394712C422F44704983522F52705A832A
:20298000822F8870282E2170322E4B815C81E416F5060CF083C097FC09C0415051095C8344
:2029A0004B8352E0450E511C840C951C8FEFE81AF80A92E0690E711C860C971C49814423A8
:2029C000C1F098014B815C814A0D5B1DB6016E0D7F1D85E492E00E9489149801A5014E0DB3
:2029E0005F1D6B817C816C0D7D1D85E492E00E9489145A815523C9F09801A5018B819C81D1
:202A0000481B590BB6016E0D7F1D85E492E00E9489149801A5014E195F096B817C816C0D97
:202A20007D1D85E492E00E9489142220C9F09801A5014E0D5F1DB6018B819C81681B790BEA
:202A400085E492E00E94891498014B815C814A0D5B1DB6016E197F0985E492E00E9489146B
:202A6000332009F492CF9801A5014E195F09B6018B819C81681B790B85E492E00E94891496
:202A80009801A5018B819C81481B590BB6016E197F0985E492E00E94891477CF0F900F90A3
:202AA0000F900F90DF91CF911F910F91FF90EF90DF90CF90BF90AF909F908F907F906F90F2
:202AC0005F904F903F902F9008952F923F924F925F926F927F928F929F92AF92BF92CF9242
:202AE000DF92EF92FF920F931F93CF93DF9300D000D000D0CDB7DEB73C016A013E832D8389
:202B0000FC82EB825801A41AB50AB7FE03C0B194A194B1088D809E80861A970A97FE03C085
:202B20009194819491088A149B045CF0902F812F0D811E819D838E839C2D8D2D6B01692FE5
:202B4000782F0C151D055CF09D818E817E836D83692F782F902F812F8601C92ED82E1601D8
:202B6000201A310A2B012D813E81421A530A57FE03C0519441945108710137FE03C03FEFCB
:202B8000E31AF30AF594E7948D819E81861797075CF5A1E0B0E0BA83A983C016D1064CF11A
:202BA000D301ED91FC910484F585E02D2B813C81A8016D817E818A149B041CF04D815E8132
:202BC000B801C3010995E418F508F7FE0AC02D813E8189819A81280F391F3E832D83E20CA2
:202BE000F31C0F5F1F4FD9CF2FEF3FEF3A832983D4CF26960FB6F894DEBF0FBECDBFDF9177
:202C0000CF911F910F91FF90EF90DF90CF90BF90AF909F908F907F906F905F904F903F90A1
:202C20002F900895EF92FF920F931F93DC011A960D911C911B9718962D913C911997ED91E1
:202C4000FC9100A0F1A1E02D7B0150E040E070E060E009951F910F91FF90EF900895EF9232
:202C6000FF920F931F93DC01ED91FC9100A0F1A1E02D780101E010E009951F910F91FF9081
:202C8000EF900895EF92FF920F931F93DC01ED91FC9100A0F1A1E02D7801890121E030E077
:202CA00009951F910F91FF90EF900895089590E080E00895009769F0FC0101900020E9F7F3
:202CC0003197AF01481B590BBC0185E492E00C94D00690E080E008959B012E503742223055
:202CE000310500F5FC0101900020E9F73197E81BF90B20917E0266E0269F900111242E9F7D
:202D0000D0012F9FB00D3E9FB00D112460914D0270914E026A1B7B0B77FF02C06F5F7F4F18
:202D200075956795709352026093510250935402409353020C945A160E943E2C1F93CF935F
:202D4000DF9385ED8093BC008091CD019091CE01A091CF01B091D0010796A11DB11D23E0B2
:202D6000B695A795979587952A95D1F72091BC0024FD03C01092150252C04091CD01509161
:202D8000CE016091CF017091D001452B462B472B69F30097A105B10541F025E32A95F1F74F
:202DA00000000197A109B109E1CF8091CC01C1E0C093CB01882399F1D091B8001091BA0020
:202DC0008091BC008A7B8093BC0060E082E10E94FD0660E083E10E94FD0610921502C093B5
:202DE00017021092160261E082E10E94FD0661E083E10E94FD068091B9008E7F8093B900CA
:202E00008091B9008D7F8093B90088E48093B80085E48093BC001093BA00D093B800DF91B9
:202E2000CF911F9108952F923F924F925F926F927F928F929F92AF92BF92CF92DF92EF9238
:202E4000FF920F931F93CF93DF93CDB7DEB7C759D2400FB6F894DEBF0FBECDBF70E060E097
:202E600085E492E00E94121680917C0290917D02E12C38EFF32EF0927B02E0927A02F092BA
:202E80005602E092550290935802809357022DE030E04FE351E070E060E090E080E00E94A6
:202EA000DF0A80917C0290917D0208E012E410937B0200937A0210935602009355029093E5
:202EC0005802809357022FEE30E04FE351E062EE70E090E080E00E94DF0A8FEF9FEF909372
:202EE0007B0280937A029093560280935502F0927D02E0927C02F0925802E092570241E028
:202F000050E06EE077E283E391E00E946C1610937D0200937C02109358020093570280EE55
:202F20009FEF90937B0280937A02909356028093550243EE50E06EE077E28BE591E00E9464
:202F40006C1680917C0290917D024FE1C42ED12CD0927B02C0927A02D0925602C092550291
:202F600090935802809357025FE1E52EF12C04ED10E020E431E04EE050E070E060E085E4AB
:202F800092E00E944011D0927B02C0927A02D0925602C092550210927D0210927C021092D9
:202FA00058021092570220EE30E04FE950E06FE070E08FE990E00E94171227E730E04EE395
:202FC00051E067E770E081E090E00E94171209E010E029E730E0A80165E770E0C8010E94DD
:202FE0001712065F1F4F0F3321E0120791F703E110E0980141EA50E0B8018DE990E00E94E8
:203000001712065F1F4F053E110599F720917C0230917D028FEF97E090937B0280937A0238
:20302000909356028093550230935802209357024FE050E065E070E083E891E00E946C168E
:2030400001E010E0B801012E000C880B990B0E945A2A27ED33EA40E95FE30E94252B23ECB1
:2030600035EF48E450E40E94252B20E030E044E353E40E94B0290E94922B20E030E04EEB49
:2030800052E40E94252B20E030E04EEE52E40E943F290E94222AC8010E94780B0F5F1F4FC4
:2030A0000E3331E0130771F620917C0230917D0280E098EF90937B0280937A02909356023D
:2030C0008093550230935802209357024BE150E065E070E087E891E00E946C1601E010E097
:2030E000B801012E000C880B990B0E945A2A27ED33EA40E95FE30E94252B23EC35EF48E492
:2031000050E40E94252B20E030E044E353E40E94B0290E94AB2920E030E04EEB52E40E9409
:20312000252B20E030E04EEE52E40E943F290E94222AC8010E94780B0F5F1F4F0E3341E099
:20314000140771F620917C0230917D0280EE9FEF90937B0280937A0290935602809355026E
:20316000309358022093570247E250E065E070E08BE891E00E946C1601E010E0B801012E77
:20318000000C880B990B0E945A2A27ED33EA40E95FE30E94252B23EC35EF48E450E40E9403
:2031A000252B20E030E044E353E40E94B0290E949A2B20E030E04EEE52E40E943F290E9441
:2031C000222AC8010E94780B0F5F1F4F0E3381E01807A1F660ED77E080E090E00E946E07F6
:2031E00080917C0290917D0210927B0210927A021092560210925502909358028093570287
:2032000020EE30E04EE351E06FE070E081E090E00E94DF0A8FE190E090937B0280937A0224
:20322000909356028093550210927D0210927C02109258021092570220EE30E04FE950E0EB
:203240006FE070E08FE990E00E94171227E730E04EE351E067E770E081E090E00E94171262
:20326000EE24E394F12C01E010E08FE1A82EB12CCC24CA9497E0D92E2CE9822E99249A9438
:203280000F5F1F4F80917C0290917D020F33E1E01E0711F40C942922F0E4EF16F1E0FF065C
:2032A00004F10F39110511F00C943222B0927B02A0927A02B0925602A092550290935802B9
:2032C00080935702F8013197EE0FFF1F81E090E08C0F9D1FE80FF91F60817181C8010E9431
:2032E000780B80917C0290917D02D0927B02C0927A02D0925602C09255029093580280937C
:203300005702B7010F2C000C880B990B0E945A2A2DEC3CEC4CE85FE30E94252B23EC35EF1C
:2033200048E450E40E94252B20E030E044E353E40E94B0290E94922B2B013C01C701B4010D
:203340000E94102C665A7F4F072E000C880B990B0E945A2AA30192010E94252B20E030E02A
:203360004EEE52E40E943F290E94222A2B01C8010E94780BF8013197EE0FFF1F21E030E0DC
:203380002C0F3D1FE20FF31F518240823FEFE31AF30A48EDE41648E1F40609F071CF60EDFE
:2033A00077E080E090E00E946E0780917C0290917D0210927B0210927A02109256021092C7
:2033C0005502909358028093570220EE30E04EE351E06FE070E081E090E00E94DF0A8AE5C3
:2033E00090E001E010E020EE422E27E0522E3FE1632E38EF732E4FE1C42ED12C50EEA52EDE
:20340000BB24BA94812C68EF962E20917C0230917D020330110509F481C30CF066C3023067
:20342000110509F472C370927B0260927A02709256026092550230935802209357027C010E
:20344000E4E1EE0EF11CAC01445C5F4FBC016852710997010E94DF0A0F5F1F4FC7010630B5
:20346000110599F660ED77E080E090E00E946E0780917C0290917D0210927B0210927A02B0
:203480001092560210925502909358028093570220EE30E04EE351E06FE070E081E090E060
:2034A0000E94DF0A72E3A72EB12CCC24C394D12CFFE12F2EF8EF3F2EAFE14A2E512CB0EE82
:2034C0008B2E99249A94612C18EF712E80917C0290917D02F3E0CF16D10409F44CC30CF051
:2034E0002FC332E0C316D10409F43CC330927B0220927A0230925602209255029093580211
:203500008093570228E131E02A193B098CED90E08A199B09B901681B790BAB014F5F5F4FA5
:2035200057FF04C0AB0140955095C901E0907A02F0907B0200917F0210E02DE330E0B50180
:203540000E9403143FEFC31AD30A44E1A40EB11C86E0C816D10409F0B9CF60ED77E080E088
:2035600090E00E946E0780917C0290917D0210927B0210927A021092560210925502909342
:2035800058028093570220EE30E04EE351E06FE070E081E090E00E94DF0A98E7A92EB12CB7
:2035A000CC24C394D12C3FE1232E38EF332E4FE1442E512C50EE852E99249A94612C68EFEF
:2035C000762E80917C0290917D02E3E0CE16D10409F400C30CF0E3C222E0C216D10409F48F
:2035E000F0C230927B0220927A0230925602209255029093580280935702E0907A02F09034
:203600007B02A5014654510987012DE330E0B50185E492E00E941C13B5016852710910E0AF
:2036200000E023E04EE150E0C5010E942813FFEFCF1ADF0A24E1A20EB11C36E0C316D1049F
:2036400009F0BFCF60ED77E080E090E00E946E0780917C0290917D0210927B0210927A02EC
:203660001092560210925502909358028093570220EE30E04EE351E06FE070E081E090E07E
:203680000E94DF0A20917C0230917D0280E098EF90937B0280937A02909356028093550235
:2036A00030935802209357020FE010E0B801012E000C880B990B0E945A2A2CEE31E548EB4E
:2036C0005FE30E94252B20E030E040E251E40E943E290E94222A20EE30E0AB01B80181E074
:2036E00090E00E9417120B5F1F4F013E1105F1F620917C0230917D0280E098EF90937B0285
:2037000080937A029093560280935502309358022093570200EE10E0B801012E000C880BA7
:20372000990B0E945A2A2CEE31E548EB5FE30E94252B20E030E040E351E40E943E290E9415
:20374000222A2FE030E0AB01B8018EE391E00E941712055011090E301105F1F620917C0213
:2037600030917D028FEF97E090937B0280937A0290935602809355023093580220935702D7
:2037800000EE10E0B801012E000C880B990B0E945A2A2CEE31E548EB5FE30E94252B9B01C7
:2037A000AC0160E070E885EA93E40E943E290E94222A2FE030E0AB01B80181E090E00E94F0
:2037C0001712055011090E301105E1F620917C0230917D028FEF97E090937B0280937A0293
:2037E000909356028093550230935802209357020FE010E0B801012E000C880B990B0E940F
:203800005A2A2CEE31E548EB5FE30E94252B9B01AC0160E070E085EA93E40E943E290E9423
:20382000222A20EE30E0AB01B8018EE391E00E9417120B5F1F4F013E1105E1F660ED77E064
:2038400080E090E00E946E0780917C0290917D0210927B0210927A02109256021092550222
:20386000909358028093570221EE30E04EE351E06FE070E081E090E00E94DF0A84E690E009
:20388000CA56DD4F99838883C659D2400E9483284B015C010E9483286B017C010E9483280B
:2038A0002B013C01C501B4012FEF30E040E050E00E94DB28162FC701B6012FEF30E040E0EF
:2038C00050E00E94DB28062FC301B2012FEF30E040E050E00E94DB28862F412F602F0E94EE
:2038E000B0060E94832820E031E040E050E00E94DB283B01E0E26E0E711C0E94832822E960
:2039000030E040E050E00E94DB287B01FDE2EF0EF11C0E9483282EE130E040E050E00E94DF
:20392000DB284B012B0100917A0210917B0221E030E0261B370BC257DD4F39832883CE587B
:20394000D24090E080E088199909FC01EE0FFF1FCE56DD4FF983E883C259D240A701480DC9
:20396000591D9801B30185E492E00E948914A701481959099801B30185E492E00E94891498
:20398000B301680D791D9801A70185E492E00E948914B301681979099801A70185E492E03A
:2039A0000E948914312C212C21E030E0CC56DD4F39832883C459D240241435040CF01EC1DD
:2039C000C257DD4F88819981CE58D24097FD1EC091E0491A5108CE56DD4FE881F981C2595A
:2039E000D2403296CE56DD4FF983E883C259D240C257DD4F28813981CE58D2402E0F3F1F0E
:203A0000C257DD4F39832883CE58D2403FEF231A330ACC56DD4F88819981C459D2400296E2
:203A2000CC56DD4F99838883C459D240C257DD4FE881F981CE58D240E80FF91FC257DD4F2E
:203A4000F983E883CE58D2404301820C931C98016701C40CD51CA601B40185E492E00E942B
:203A600089145301A218B3089801A601B50185E492E00E94891498016701C418D508A6016F
:203A8000B40185E492E00E9489149801A601B50185E492E00E9489146701C20CD31C980189
:203AA000A6015301A40CB51CB50185E492E00E9489149801A6016301C418D508B60185E43D
:203AC00092E00E9489144701821893089801A401B50185E492E00E9489149801A401B601B5
:203AE00085E492E00E94891467CF04301105F9F00530110509F097CCB0927B02A0927A022F
:203B0000B0925602A092550296CC90927B0280927A0290925602809255028DCC50927B0258
:203B200040927A02509256024092550284CCD0927B02C0927A02D0925602C09255027BCC2D
:203B400044E0C416D10411F1E5E0CE16D10409F0CDCC90927B0280927A02909256028092C7
:203B60005502CCCC70927B0260927A027092560260925502C3CC20EE37E030937B0220931F
:203B80007A023093560220935502B8CC50927B0240927A025092560240925502AFCC34E061
:203BA000C316D10411F145E0C416D10409F019CD90927B0280927A02909256028092550292
:203BC00018CD70927B0260927A0270925602609255020FCDE0EEF7E0F0937B02E0937A0200
:203BE000F0935602E093550204CD50927B0240927A025092560240925502FBCCCA56DD4F2C
:203C000028813981C659D24021503109CA56DD4F39832883C659D240232B09F037CE60EDE8
:203C200077E080E090E00E946E0780917C0290917D0210927B0210927A021092560210923E
:203C40005502909358028093570220EE30E04EE351E06FE070E081E090E00E94DF0A14E6AF
:203C6000212E312C412C512C32014A940E9483284B015C010E9483286B017C010E94832824
:203C8000C257DD4F688379838A839B83CE58D240C501B401A30192010E94DB28162FC70131
:203CA000B601A30192010E94DB28062FC257DD4F688179818A819B81CE58D240A30192017E
:203CC0000E94DB28862F412F602F0E94B0060E9483282CE331E040E050E00E94DB286B0165
:203CE00032E0C30ED11C0E9483282FEC30E040E050E00E94DB285B0140E1A40EB11C0E94E9
:203D000083282CE331E040E050E00E94DB287B01E2E0EE0EF11C0E9483282FEC30E040E004
:203D200050E00E94DB28605F7F4FA7014C195D099A012F5F3F4FCB018A199B098C010F5FE9
:203D40001F4F37FF04C09A0120953095670117FF04C08C01009510955B01E0907A02F09015
:203D60007B02A501B60185E492E00E944011F1E02F1A310809F07ACF60ED77E080E090E092
:203D80000E946E0780917C0290917D0210927B0210927A0210925602109255029093580230
:203DA0008093570220EE30E04EE351E06FE070E081E090E00E94DF0A24E630E0C257DD4FBD
:203DC00039832883CE58D2400E9483284B015C010E9483286B017C010E9483282B013C0162
:203DE000C501B4012FEF30E040E050E00E94DB28162FC701B6012FEF30E040E050E00E9441
:203E0000DB28062FC301B2012FEF30E040E050E00E94DB28862F412F602F0E94B0060E9422
:203E200083282CE331E040E050E00E94DB283B0132E0630E711C0E9483282FEC30E040E0DE
:203E400050E00E94DB281B0140E1240E311C0E9483282CE331E040E050E00E94DB288B01E3
:203E60000E5F1F4F0E9483282FEC30E040E050E00E94DB28605F7F4F9801261937095901FB
:203E80008FEFA81AB80ACB01821993096C01EFEFCE1ADE0AB7FE04C05901A094B09438017E
:203EA000D7FE04C06C01C094D0941B0140907A0250907B02E0907F02F12CAC14BD042CF4D0
:203EC000C501B7FE05C0019603C0C601D7FCFBCF959587958E159F050CF47C019701220F11
:203EE000331FCE56DD4F39832883C259D240C501821B930BCC56DD4F99838883C459D240E7
:203F00004701860C971C82019C01A101B40185E492E00E941013F101EC0DFD1DCA56DD4FAC
:203F2000F983E883C659D240AF0141505109CC56DD4F28813981C459D240B40185E492E05E
:203F40000E941013CE56DD4F28813981C259D240C21AD30A2E0C3F1C9601A101B30185E418
:203F600092E00E941C13A60CB71CB501615071099601A10185E492E00E941C1321E0A7010A
:203F8000B101C4010E949014AE18BF0831E0A31AB10822E0A701B101C5010E949014CA56C8
:203FA000DD4FC880D980C659D240CE18DF0841E0C41AD10824E0A701B601C5010E949014EF
:203FC00028E0A701B601C4010E949014C257DD4F88819981CE58D2400197C257DD4F9983D6
:203FE0008883CE58D240892B09F0EECE60ED77E080E090E00E946E0780917C0290917D025B
:2040000010927B0210927A021092560210925502909358028093570220EE30E04EE351E007
:204020006FE070E081E090E00E94DF0AF4E62F2E312C0E9483284B015C010E9483286B0142
:204040007C010E9483282B013C01C501B4012FEF30E040E050E00E94DB28162FC701B601CB
:204060002FEF30E040E050E00E94DB28062FC301B2012FEF30E040E050E00E94DB28862F99
:20408000412F602F0E94B0060E9483284B015C010E9483282B013C010E9483286B017C01E7
:2040A0000E94832821ED30E040E050E00E94DB28FB017096C257DD4FF983E883CE58D2403A
:2040C000C701B6012CE331E040E050E00E94DB287B01F2E0EF0EF11CC301B20121ED30E05F
:2040E00040E050E00E94DB288B01005F1F4FC501B4012CE331E040E050E00E94DB28CB0116
:204100000296C257DD4F28813981CE58D240A701B8010E94171221E0221A310809F089CF34
:2041200060ED77E080E090E00E946E0780917C0290917D0210927B0210927A02109256028E
:2041400010925502909358028093570220EE30E04EE351E06FE070E081E090E00E94DF0A02
:2041600070E1272E77E2372EC12CD12C7601CA940E9483282B013C010E9483284B015C0170
:204180000E948328C257DD4F688379838A839B83CE58D240C301B201A70196010E94DB28E8
:2041A000162FC501B401A70196010E94DB28062FC257DD4F688179818A819B81CE58D2409F
:2041C000A70196010E94DB28862F412F602F0E94B0060E9483282B013C010E9483284B01A0
:2041E0005C01C301B20121ED30E040E050E00E94DB288B01005F1F4FC501B4012CE331E0E4
:2042000040E050E00E94DB28CB010296B8010E94780B31E0231A310809F0AACF60ED77E0CA
:2042200080E090E00E946E076FE170E085E492E00E94121680917C0290917D02C12C58EFEF
:20424000D52ED0927B02C0927A02D0925602C0925502909358028093570200917F0210E060
:20426000E12C68EFF62E24E630E040EA50E066E470E080E590E00E9403148FEF9FEF9093EB
:204280007B0280937A029093560280935502D0927D02C0927C02D0925802C09257024DE5E3
:2042A00050E06EE077E28FE891E00E946C1647E750E06EE077E28AE991E00E946C1644E8E2
:2042C00050E06EE077E28AEA91E00E946C1680EE97E090937B0280937A029093560280935C
:2042E00055028FE190E090937D0280937C02909358028093570242ED50E06EE077E289EBF1
:2043000091E00E946C168FB7F89480903C0290903D02A0903E02B0903F028FBFC357DD4F04
:204320001882CD58D24081149104A104B104D1F1D501C401B7FE07C088279927DC01881962
:204340009909AA09BB09BC01CD010DE712E00C0F1D1F005F1F4F3AE0432E512C612C712C7D
:204360004DE7E42E42E0F42EEC0EFD1E46E0E40EF11CA30192010E94DB28605DF8016293F2
:204380008F01B901CA01611571058105910519F00E151F0571F7B7FE11C0F8018DE2829345
:2043A0008F010CC080E3C457DD4F8883CC58D2400DE712E00C0F1D1F015F1F4FF801019021
:2043C0000020E9F73197E01BF10B80917E0226E0829FC00111248E9F90018F9F300D9E9F0A
:2043E000300D112480914D0290914E02821B930B97FD0196959587959093520280935102F1
:2044000081EE90E09093540280935302C8010E945A1660E177E280E090E00E946E07C95661
:20442000DD4F0FB6F894DEBF0FBECDBFDF91CF911F910F91FF90EF90DF90CF90BF90AF907F
:204440009F908F907F906F905F904F903F902F90089501E010E030E4E31631E0F30614F417
:204460000C947119F8013197EE0FFF1F21E030E02C0F3D1FE20FF31F2081318127373105A4
:2044800011F40C94561910927B0210927A0210925602109255020C945E191F920F920FB6AA
:2044A0000F9211242F933F938F939F93AF93BF9380913C0290913D02A0913E02B0913F0208
:2044C00030913B0223E0230F2D3758F50196A11DB11D20933B0280933C0290933D02A093FF
:2044E0003E02B0933F028091400290914102A0914202B09143020196A11DB11D80934002CE
:2045000090934102A0934202B0934302BF91AF919F918F913F912F910F900FBE0F901F900C
:20452000189526E8230F0296A11DB11DD2CF1F920F920FB60F9211242F933F934F935F9374
:204540006F937F938F939F93AF93BF93EF93FF938091B900887F803609F44AC0F0F588321E
:2045600009F4A5C018F5803109F499C0B8F4882309F4F5C0883009F492C0FF91EF91BF9155
:20458000AF919F918F917F916F915F914F913F912F910F900FBE0F901F901895883109F4FE
:2045A00086C0803251F78093140214C0803409F49BC040F48033B9F38833F9F6809314024C
:2045C00085ECAEC0803509F483C0883509F494C0883499F60E949E16D0CF883909F48AC0B1
:2045E00038F5883729F050F4883611F0803729F683E0809315021092130255C0883809F4C7
:2046000079C0803919F0803809F0B7CF80911302803208F06FC0E091130281E08E0F8093D2
:2046200013028091BB00F0E0ED50FE4F80833BC0803B39F0D0F4803A09F477C0883A09F0F0
:204640009CCF84E0809315021092F2011092F101F0E0E0E009958091F10181110FC081E045
:204660008093F1011092D10109C0803C09F4A8CF883C09F4A5CF883B09F07FCFE091F20125
:2046800081E08E0F8093F201F0E0EF52FE4F80818093BB009091F2018091F10129C08091D8
:2046A0003A028093BB0085EC8093BC0066CF9091390280913802981758F5E091390281E0CB
:2046C0008E0F80933902F0E0E85EFD4F8081E9CFE091390281E08E0F809339028091BB0010
:2046E000F0E0E85EFD4F808390913902809138029817C8F285E8D8CFE091390281E08E0F87
:20470000809339028091BB00F0E0E85EFD4F80838091170281115ECF81E08093160284EA37
:204720008093BC001092150228CF85EC8093BC001092150280911302803230F4E09113027F
:20474000F0E0ED50FE4F10826091130270E083EF91E0F0E0E0E00995109213020ECF1092D0
:20476000140238CFE5E4F2E01382128220EF30E03583248380E491E0978386833187208783
:2047800093878287168A158614861786168681E0858B848B2FEF3FEF338B228B318B208B4A
:2047A000878B108E128E118E8BE091E0918380830895CF93DF9300D01F92CDB7DEB7789400
:2047C00084B5826084BD84B5816084BD85B5826085BD85B5816085BD80916E0081608093F4
:2047E0006E00109281008091810082608093810080918100816080938100809180008160A7
:20480000809380008091B10084608093B1008091B00081608093B00080917A0084608093B4
:204820007A0080917A00826080937A0080917A00816080937A0080917A00806880937A000B
:204840001092C10085E480937C0080917A00806480937A0080917A0086FDFCCF809178009F
:2048600060917900762F682F072E000C880B990B611571058105910511F00E94D228E4EFA2
:20488000F5E02491E0EEF5E08491882399F090E0880F991FFC01E853FA4FA591B491FC01EA
:2048A000E254FA4F859194918FB7F894EC91E22BEC938FBF61E08EE00E94FD060E94A10777
:2048C00060E090E080E00E94CD077C018830944521F180E2E81684E5F806F9F029E8E21679
:2048E000F20609F4ABC360E087E690E00E94CD078734974409F4A7C381EA90E00E941C0824
:20490000613081E6780709F4A3C36F3F7F4F09F045C0A6E2EA2EA5E1FA2E0E94A107109209
:20492000610210926002F0926502E092640222E0E21623E9F20609F446C308F0A2C120E1EF
:20494000E21623E5F20609F4B9C208F037C120E2E21625E1F20609F497C208F009C125E0E2
:20496000E21625E1F20609F428C281E1E81685E1F80609F42DC224E5E21621E0F20609F0B7
:2049800004C182E090E190936302809362026CE970E08AEF9BE00E946F08F7C08FEB90E02D
:2049A0000E943B087B0187E5E81683E8F80609F4B4CF21E8E21624E9F20609F4AECF81E161
:2049C000E81685E1F80609F4A8CF20E2E21625E1F20609F4A2CF86E2E81685E1F80609F4D4
:2049E00098CF21E8E21625E1F20609F496CFE11484E1F80609F431C384ED90E00E941C08FF
:204A00007B016031734509F488CF8FEE90E00E943B087B0187E2E81683E9F80609F47DCF15
:204A200084E090E00E941C087B01811121C061157048F1F48091040190910501A091060165
:204A400089839A83AB83AE014F5F5F4F63E089EB90E00E94C90860E080ED90E00E94CD07C7
:204A6000893911F08039B1F4F0E9EF2EFE2C55CF86E2E81685E1F80609F44BCF22E5E216F1
:204A800025E8F20609F4EEC281E1E8168CEAF80609F443CF83ED90E00E941C08872FE62E11
:204AA000F72E8359823008F450C0783909F44DC0773709F44AC0763109F447C023EDE21614
:204AC000F104C9F5E0E9EE2EFE2C0E94A1071092610210926002E114F10409F024CF81E486
:204AE00093E9909365028093640283E194E0909363028093620283ED90E00E941C0805E6CF
:204B000010E056EDE52E56E0F52E672B682B692B09F076C18091620290916302846090613D
:204B2000909363028093620202E210E0F9E0EF2EF6E0FF2E65C183EDE816F80619F260E0CC
:204B400090E080E00E94CD077C01E114F10459F023EDE216F10409F4B5CF83EDE816F80675
:204B600009F0B3CFAFCF71E4E72E73E9F72EADCF81E8E81685E1F80609F428C248F486E27F
:204B8000E81685E1F80609F48CC1F12CE12C38C122E0E21626E1F20609F412C285E3E81616
:204BA00085E4F80691F780E090E190936302809362026CE970E08EE59BE0EDCE29E8E216DF
:204BC00027E7F20609F4ACC170F529E0E21628E6F20609F4CBC180F484E091E128E0E21626
:204BE00024E5F20691F6909363028093620268ED70E086EF99E0CFCE84E1E81688E6F8062F
:204C000009F475C123E8E21627E7F20609F0BDCF82E091E1909363028093620260E970E067
:204C20008EEC9AE0B8CE86E9E81687E7F80609F4E9C1C8F483E9E81687E7F80609F0A5CF7B
:204C400080E090E1909363028093620260EC70E08AEB97E00E946F0880E991E090934C0298
:204C600080934B0292CF27E5E21623E8F20609F464C180E9E816F80609F087CF83E194E1BD
:204C80005EC122E4E21623E9F20608F041C080E4E81683E9F80608F028CF28E2E21623E931
:204CA000F20609F46EC1A8F425E2E21623E9F20609F467C187E2E81683E9F80609F467C116
:204CC00020E2E21623E9F20609F05FCF84E090E18ACF81E3E81683E9F80609F455C148F466
:204CE00089E2E81683E9F80609F04FCF83E096E14DC025E3E21623E9F20609F445C188E371
:204D0000E81683E9F80609F040CF83E194E03EC029E8E21624E9F20658F587E8E81684E918
:204D2000F80608F088C121E8E21624E9F20609F466C186E8E81684E9F80609F026CF83E0E2
:204D400094E1909363028093620280EE91E090934C0280934B0280E491E090934A028093D8
:204D600049020BE310E076E5E72E76E0F72E48C025E0E21625EBF20601F198F483E194E1BB
:204D800021E1E2162CEAF20609F0FFCE909363028093620203E010E0ABE3EA2EA7E0FA2E1E
:204DA0002FC089E0E81685EBF80609F449CF25E0E21625ECF20609F0E8CE88E090E1909369
:204DC00063028093620260EB70E08AE798E0E3CD83E090E0909363028093620280EE91E012
:204DE00090934C0280934B0280E491E090934A028093490203E010E067EBE62E67E0F62E9C
:204E000020916302822F82958F7090E0817099279093670280936602E114F10481F069E0E9
:204E200070E080E096E00E94F508B801C7010E94F50866E070E08AEF95E00E94F50860E02A
:204E400085E492E00E94820B60E085E492E00E94420911E01093800261E085E492E00E946C
:204E6000820B84E080937F0210937E021093590210935A0200E010E00E94131701151105C5
:204E8000D9F30E940000F8CF83E194E0909363028093620206E010E051EBE52E57E0F52E87
:204EA000AFCF83E194E090936302809362020CE010E045EAE42E47E0F42EA2CF83E19EE0E4
:204EC000909363028093620280EE91E090934C0280934B0280E491E090934A028093490281
:204EE00002E010E033EAE32E37E0F32E89CF83E094E0909363028093620280EE91E090934A
:204F00004C0280934B0280E491E090934A028093490203E010E020EAE22E27E0F22E70CFEE
:204F200083E194E0909363028093620201E410E09FE5E92E97E0F92E63CF83E094E190935F
:204F400063028093620280EE91E090934C0280934B0280E491E090934A028093490203E040
:204F600010E08CE5E82E87E0F82E4ACF82E091E190936302809362026CEC70E08AE299E0B4
:204F80000ACD80E091E1F4CF80E090E1F1CF83E094E0909363028093620280E991E0909341
:204FA0004C0280934B0280EF90E090934A02809349020EE110E0BEE3EB2EB7E0FB2E20CF4F
:204FC00083E195E0E3CE83E094E0E0CE83E194E0909363028093620280EE91E090934C029B
:204FE00080934B0280E491E090934A028093490205E410E0E1E9EE2EE6E0FE2E01CF87E0C7
:2050000094E0E6CF83E094E0909363028093620280EE91E090934C0280934B0280E491E00C
:2050200090934A02809349020BE210E06BE2E62E66E0F62EE5CE83E194E0E6CF49E8E42E78
:2050400042E1F42E6ACC37E4E32E33E8F32E65CC23E6E22E29E1F22E60CC94E1E92E98E6C3
:20506000F92E5BCC89E8E82E87E7F82E56CC8F929F92AF92BF92CF92DF92EF92FF92CF937B
:20508000DF93EC01688179818A819B81611571058105910521F464E279ED8BE597E02DE1E9
:2050A00033EF41E050E00E94DB2849015A019B01AC01A7EAB1E40E94FA286B017C01ACEE7D
:2050C000B4EFA50194010E940829C60ED71EE81EF91EF7FE06C081E0C81AD108E10880E811
:2050E000F80AC882D982EA82FB82C701B6019F77DF91CF91FF90EF90DF90CF90BF90AF9051
:205100009F908F9008958F929F92AF92BF92CF92DF92EF92FF9260910001709101018091D6
:20512000020190910301611571058105910521F464E279ED8BE597E02DE133EF41E050E016
:205140000E94DB2849015A019B01AC01A7EAB1E40E94FA286B017C01ACEEB4EFA501940171
:205160000E940829C60ED71EE81EF91EF7FE06C081E0C81AD108E10880E8F80AC0920001F9
:20518000D0920101E0920201F0920301C701B6019F77FF90EF90DF90CF90BF90AF909F9082
:2051A0008F900895609300017093010180930201909303010895052E97FB1EF400940E9453
:2051C000F22857FD07D00E940D2907FC03D04EF40C94F22850954095309521953F4F4F4F7F
:2051E0005F4F089590958095709561957F4F8F4F9F4F08950E942F29A59F900DB49F900D2D
:20520000A49F800D911D11240895B7FF0C94FA280E94FA28821B930B0895A1E21A2EAA1B9A
:20522000BB1BFD010DC0AA1FBB1FEE1FFF1FA217B307E407F50720F0A21BB30BE40BF50B2B
:20524000661F771F881F991F1A9469F760957095809590959B01AC01BD01CF010895A29FDD
:20526000B001B39FC001A39F700D811D1124911DB29F700D811D1124911D08955058BB27B4
:20528000AA270E9456290C94D72A0E949E2A38F00E94A52A20F039F49F3F19F426F40C9496
:2052A0009B2A0EF4E095E7FB0C94952AE92F0E94FC2A58F3BA17620773078407950720F05B
:2052C00079F4A6F50C941E2B0EF4E0950B2EBA2FA02D0B01B90190010C01CA01A001112472
:2052E000FF27591B99F0593F50F4503E68F11A16F040A22F232F342F4427585FF3CF469523
:2053000037952795A795F0405395C9F77EF41F16BA0B620B730B840BBAF09150A1F0FF0FE1
:20532000BB1F661F771F881FC2F70EC0BA0F621F731F841F48F4879577956795B795F79593
:205340009E3F08F0B0CF9395880F08F09927EE0F9795879508950E94AE2AE3950C94E82AFC
:205360000E94C4290C94D72A0E94A52A58F00E949E2A40F029F45F3F29F00C94952A511115
:205380000C941F2B0C949B2A0E94FC2A68F39923B1F3552391F3951B550BBB27AA27621703
:2053A0007307840738F09F5F5F4F220F331F441FAA1FA9F335D00E2E3AF0E0E832D09150B3
:2053C0005040E695001CCAF72BD0FE2F29D0660F771F881FBB1F261737074807AB07B0E824
:2053E00009F0BB0B802DBF01FF2793585F4F3AF09E3F510578F00C94952A0C941F2B5F3F16
:20540000E4F3983ED4F3869577956795B795F7959F5FC9F7880F911D9695879597F90895A6
:20542000E1E0660F771F881FBB1F621773078407BA0720F0621B730B840BBA0BEE1F88F7F5
:20544000E09508950E94292A6894B1110C941F2B08950E94042B88F09F5798F0B92F992791
:20546000B751B0F0E1F0660F771F881F991F1AF0BA95C9F714C0B13091F00E941E2BB1E07E
:2054800008950C941E2B672F782F8827B85F39F0B93FCCF3869577956795B395D9F73EF436
:2054A00090958095709561957F4F8F4F9F4F0895E89409C097FB3EF4909580957095619542
:2054C0007F4F8F4F9F4F9923A9F0F92F96E9BB279395F695879577956795B795F111F8CF68
:2054E000FAF4BB0F11F460FF1BC06F5F7F4F8F4F9F4F16C0882311F096E911C0772321F0D0
:205500009EE8872F762F05C0662371F096E8862F70E060E02AF09A95660F771F881FDAF76C
:20552000880F9695879597F9089597F99F6780E870E060E008959FEF80EC089500240A94DC
:205540001616170618060906089500240A94121613061406050608950C949B2A0E94042B3D
:20556000D8F3E894E0E0BB279F57F0F02AED3FE049EC06C0EE0FBB0F661F771F881F28F09A
:20558000B23A62077307840728F0B25A620B730B840BE3959A9572F7803830F49A95BB0F2E
:2055A000661F771F881FD2F790480C94C12B092E0394000C11F4882352F0BB0F40F4BF2B48
:2055C00011F460FF04C06F5F7F4F8F4F9F4F0895EF93E0FF07C0A2EA2AED3FE049EC5FEB35
:2055E0000E9456290E94D72A0F90039401FC9058E8E6F0E00C94CD2B57FD9058440F551F93
:2056000059F05F3F71F04795880F97FB991F61F09F3F79F087950895121613061406551F65
:20562000F2CF4695F1DF08C0161617061806991FF1CF86957105610508940895E894BB27C9
:2056400066277727CB0197F908950E94382B0C94D72A0E949E2A38F00E94A52A20F09523B5
:2056600011F00C94952A0C949B2A11240C941F2B0E94FC2A70F3959FC1F3950F50E0551FEB
:20568000629FF001729FBB27F00DB11D639FAA27F00DB11DAA1F649F6627B00DA11D661F63
:2056A000829F2227B00DA11D621F739FB00DA11D621F839FA00D611D221F749F3327A00DCE
:2056C000611D231F849F600D211D822F762F6A2F11249F5750409AF0F1F088234AF0EE0F45
:2056E000FF1FBB1F661F771F881F91505040A9F79E3F510580F00C94952A0C941F2B5F3F55
:20570000E4F3983ED4F3869577956795B795F795E7959F5FC1F7FE2B880F911D9695879533
:2057200097F908959F930E94AE2A0F9007FCEE5F0C94E82ADF93D92F0E94AE2AE695D79514
:205740002AED3FE049E45FE3B33A6207730784079507D7953AF0A2EA49EC90680E9456293D
:205760000E94D72AE6E8F0E00E94CD2BDD0F13F00E94E12BDD0F0BF49058DF9108959F3FF3
:2057800031F0915020F4879577956795B795880F911D9695879597F908959F938F937F9364
:2057A0006F93FF93EF939B01AC010E94252BEF91FF910E94E92B2F913F914F915F910C94D2
:2057C000252B9B01AC0160E070E080E89FE30C94B029DF93CF931F930F93FF92EF92DF9292
:2057E0007B018C01689406C0DA2EEF010E94382BFE01E894A5912591359145915591A6F35F
:20580000EF010E945629FE019701A801DA9469F7DF90EF90FF900F911F91CF91DF9108952F
:2058200097FB072E16F4009407D077FD09D00E94242C07FC05D03EF4909581959F4F08951D
:20584000709561957F4F0895AA1BBB1B51E107C0AA1FBB1FA617B70710F0A61BB70B881F06
:20586000991F5A95A9F780959095BC01CD010895EE0FFF1F0590F491E02D099481E090E0CF
:20588000F8940C94432CF894FFCF01000000FF8357000000006E10D006571656160F0BAF43
:2058A00006891400131C1310136515AF06820B420942162F16290A12169F1140112A205541
:2058C0006E6976657273616C20436F6C6F722054465420446973706C6179204C6962726137
:2058E0007279202A003C687474703A2F2F656C656374726F6E6963732E68656E6E696E672F
:205900006B61726C73656E2E636F6D3E0053696E00436F730054616E00546861742773202F
:205920006974210052657374617274696E6720696E206100666577207365636F6E64732E4F
:205940002E2E0052756E74696D653A20286D736563732900FFFFFFFFFFFFFFFFFFFFFFFF4D
:20596000FFFFFFFFFFFFFFFFFFFFFFFFFFFFFFFFFFFFFFFFFFFFFFFFFFFFFFFFFFFFFFFF47
:20598000A91B3BCAD0FCD0CFF12CE12C00E310E02BE330E045E150E066EE70E0C1CF91E0BD
:2059A0009D1548F30E94C513E6CFC4018B5691094F9758F40E9450138091560291E08927CA
:2059C0008093560288E893E120CAC401885991094F9708F0E4C080914C028330E1F40E9443
:2059E0007D1380910201873120F48F5F8093020102C0109202010E94501380915E028230A4
:205A000009F0FBC98091020185508C3008F4F5C910925E02F2C9883009F040C080914D029C
:205A200090914E02019690934E0280934D024F9734F08EE190E090934E0280934D028091BA
:205A40004D02880F880F8CAF1BAE6BAC7CACB301770C880B990BE0915D0204E0E09FF001F4
:205A60001124E659FE4F20813181428153810E94183080915F0290916002280F391F30934A
:205A8000600220935F028FEF93E0211534400CF499CF9093600280935F0294CF893009F07F
:205AA00040C080914D0290914E02019690934E0280934D024F9734F08EE190E090934E024D
:205AC00080934D0280914D02880F880F8EAF1DAE6DAC7EACB301770C880B990BE091590251
:205AE00004E0E09FF0011124E659FE4F20813181428153810E94183080915B0290915C02D0
:205B0000280F391F30935C0220935B028FEF93E0211534400CF456CF90935C0280935B0214
:205B200051CF863009F04ECF80914D0290914E02019690934E0280934D0280910301A10185
:205B4000481B510910E000E02CE231E070E060E087E297E00E94A51580914D029091030148
:205B6000890F80930301A101481B510900EE1FEF2CE231E070E060E087E297E00E94A51530
:205B8000F12CE12C00E110E020E330E041E050E060EC70E087E297E00E94830F2EC965ECAE
:205BA000861A910873E28716910408F0B7C080914C02833051F40E947D138091020188236E
:205BC00011F0815013CF87E111CF883009F040C080914D0290914E02019690934E0280932A
:205BE0004D024F9734F08EE190E090934E0280934D0280914D02880F880F21968FAF21975D
:205C00001FAE21966EAC7FAC2197B301770C880B990BE0915D0204E0E09FF0011124E659FD
:205C2000FE4F20813181428153810E94183080915F0290916002821B930B9093600280937B
:205C40005F0281309C4F0CF0BDCE81E09CEF21CF893009F042C080914D0290914E020196C8
:205C600090934E0280934D024F9734F08EE190E090934E0280934D0280914D02880F880F03
:205C800023968FAF239722961FAE229723966EAC7FAC2397B301770C880B990BE091590223
:205CA00004E0E09FF0011124E659FE4F20813181428153810E94183080915B0290915C020E
:205CC000821B930B90935C0280935B0281309C4F0CF078CE81E09CEF1FCF863009F072CEF1
:205CE00080914D0290914E02019690934E0280934D0280910301A101481B510910E000E023
:205D00002CE231E070E060E087E297E00E94A5158091030190914D02891B23CFC901CD974F
:205D20008F329105E0F400321105CCF480915D02843090F48F5F80935D02F12CE12C00E11D
:205D400010E020E330E041E050E06CE370E087E297E00E94830F36CE10925D02EECFB901C0
:205D6000615071096F32710508F050C00032110534F580915E0281110EC081E080935E02C3
:205D8000F12CE12C00E110E020E330E041E050E061E070E0FFCE813079F480915A02823009
:205DA00059F08091020185508C3030F482E080935E020E945013E4CF10925E02E1CF013D54
:205DC0001105E4F180915A0281110CC081E080935A02F12CE12C00E110E020E330E040EE01
:205DE00050E0D6CF813061F480915E02823041F082E080935A0210924B020E945013E9CFF7
:205E000010925A0281E080934B02E3CF8F97B0F4013D11059CF080915902843060F48F5F05
:205E200080935902F12CE12C00E110E020E330E040EE50E08ACF10925902F4CFB9016558F8
:205E400071096F32710570F4003211055CF480914C02833019F410924C02B4CD83E08093AF
:205E60004C0250C0C901815C91098F329105E0F500321105CCF580914C02863031F5109271
:205E80004C0280910301A101481B510910E000E02CE231E070E060E087E297E00E94A51585
:205EA000F12CE12C00E110E020E330E041E050E060EC70E087E297E00E94830F20E330E0C0
:205EC00041E050E06CEF70E065CE80910201813138F786E080934C0280910301A101481BBD
:205EE000510900EE1FEFD4CF2D5F31092F323105F0F400321105DCF480914C02893089F4BB
:205F000010924C02F12CE12C00E110E020E330E041E050E060EC70E087E297E00E94830F82
:205F2000BBCC883011F489E09ACF88E098CF6F327105C0F4013D11050CF444CD8091040136
:205F4000863071F487E080930401F12CE12C00E110E024E230E040EE50E064E870E0F7CED7
:205F600086E0F1CF8F97C8F4013D11050CF42ACD8091570281110EC081E080935702F12C1A
:205F8000E12C00E110E02CE030E040EE50E060EC70E0DDCE10925702F2CF2F32310508F017
:205FA00011CD013D11050CF40DCD809158028330E0F48F5F80935802F12CE12C00E110E08D
:205FC00020E330E040EE50E06CEF70E087E297E00E94830F20E330E041E050E06CEF70E082
:205FE00087E297E00E94830FCACC1092580281E080930101E1CFFB01DC0105900D920020A8
:20600000E1F70895F999FECF92BD81BDF89A992780B50895262FF999FECF1FBA92BD81BDE1
:2060200020BD0FB6F894FA9AF99A0FBE01960895052E97FB1EF400940E942F3057FD07D073
:206040000E944A3007FC03D04EF40C942F3050954095309521953F4F4F4F5F4F089590953C
:206060008095709561957F4F8F4F9F4F08950E946C30A59F900DB49F900DA49F800D911D4C
:2060800011240895B7FF0C9437300E943730821B930B0895A1E21A2EAA1BBB1BFD010DC05F
:2060A000AA1FBB1FEE1FFF1FA217B307E407F50720F0A21BB30BE40BF50B661F771F881F7C
:2060C000991F1A9469F760957095809590959B01AC01BD01CF010895A29FB001B39FC0014D
:2060E000A39F700D811D1124911DB29F700D811D1124911D08955058BB27AA270E949330B4
:206100000C940D320E94FF3138F00E94063220F039F49F3F19F426F40C94FC310EF4E09546
:20612000E7FB0C94F631E92F0E941E3258F3BA17620773078407950720F079F4A6F50C94CE
:2061400040320EF4E0950B2EBA2FA02D0B01B90190010C01CA01A0011124FF27591B99F03F
:20616000593F50F4503E68F11A16F040A22F232F342F4427585FF3CF469537952795A795F3
:20618000F0405395C9F77EF41F16BA0B620B730B840BBAF09150A1F0FF0FBB1F661F771F22
:2061A000881FC2F70EC0BA0F621F731F841F48F4879577956795B795F7959E3F08F0B0CFA6
:2061C0009395880F08F09927EE0F9795879508950E94D23108F481E008950E9401310C9453
:2061E0000D320E94063258F00E94FF3140F029F45F3F29F00C94F63151110C9441320C948C
:20620000FC310E941E3268F39923B1F3552391F3951B550BBB27AA2762177307840738F03F
:206220009F5F5F4F220F331F441FAA1FA9F335D00E2E3AF0E0E832D091505040E695001C2A
:20624000CAF72BD0FE2F29D0660F771F881FBB1F261737074807AB07B0E809F0BB0B802D50
:20626000BF01FF2793585F4F3AF09E3F510578F00C94F6310C9441325F3FE4F3983ED4F3EE
:20628000869577956795B795F7959F5FC9F7880F911D9695879597F90895E1E0660F771FC0
:2062A000881FBB1F621773078407BA0720F0621B730B840BBA0BEE1F88F7E09508950E947F
:2062C00066316894B1110C94413208950E94263288F09F5798F0B92F9927B751B0F0E1F0A8
:2062E000660F771F881F991F1AF0BA95C9F714C0B13091F00E944032B1E008950C94403291
:20630000672F782F8827B85F39F0B93FCCF3869577956795B395D9F73EF4909580957095EE
:2063200061957F4F8F4F9F4F0895E89409C097FB3EF490958095709561957F4F8F4F9F4F58
:206340009923A9F0F92F96E9BB279395F695879577956795B795F111F8CFFAF4BB0F11F4B6
:2063600060FF1BC06F5F7F4F8F4F9F4F16C0882311F096E911C0772321F09EE8872F762F1D
:2063800005C0662371F096E8862F70E060E02AF09A95660F771F881FDAF7880F96958795E1
:2063A00097F90895990F0008550FAA0BE0E8FEEF16161706E807F907C0F012161306E4071E
:2063C000F50798F0621B730B840B950B39F40A2661F0232B242B252B21F408950A2609F495
:2063E000A140A6958FEF811D811D089597F99F6780E870E060E008959FEF80EC0895002444
:206400000A941616170618060906089500240A9412161306140605060895092E0394000C2C
:2064200011F4882352F0BB0F40F4BF2B11F460FF04C06F5F7F4F8F4F9F4F089557FD905819
:20644000440F551F59F05F3F71F04795880F97FB991F61F09F3F79F08795089512161306DE
:206460001406551FF2CF4695F1DF08C0161617061806991FF1CF869571056105089408954B
:20648000E894BB2766277727CB0197F908950E94D23108F48FEF08950E945F320C940D32AC
:2064A0000E94FF3138F00E94063220F0952311F00C94F6310C94FC3111240C9441320E94C1
:2064C0001E3270F3959FC1F3950F50E0551F629FF001729FBB27F00DB11D639FAA27F00D59
:2064E000B11DAA1F649F6627B00DA11D661F829F2227B00DA11D621F739FB00DA11D621F01
:20650000839FA00D611D221F749F3327A00D611D231F849F600D211D822F762F6A2F112421
:206520009F5750409AF0F1F088234AF0EE0FFF1FBB1F661F771F881F91505040A9F79E3FE0
:20654000510580F00C94F6310C9441325F3FE4F3983ED4F3869577956795B795F795E79512
:206560009F5FC1F7FE2B880F911D9695879597F90895FA01EE0FFF1F309621053105A1F1B9
:206580006115710561F48038BFE39B0749F168949038810561F08038BFEF9B0741F09923F4
:2065A0004AF5FF3FE1053105210519F1E8940894E795D901AA2329F4AB2FBE2FF85FD0F3D9
:2065C00010C0FF5F70F4A695E0F7F73950F019F0FF3A38F49F779F930DD00F9007FC90588A
:2065E000089546F00C94FC3160E070E080E89FE308954FE79F775F934F933F932F930E948E
:2066000014342F913F914F915F910E944C320C945C3319F416F40C94FC310C948E330E949C
:206620002632B8F39923C9F3B6F39F57550B87FF0E949C330024A0E640EA900180585695C1
:20664000979528F4805C660F771F881F20F026173707480730F4621B730B840B2029312939
:206660004A2BA69517940794202531254A2758F7660F771F881F20F026173707480730F419
:20668000620B730B840B200D311D411DA09581F7B901842F9158880F9695879508950E9487
:2066A000D231880B990B089529F416F00C94F6310C9440320C94FC310E942632A8F39638D7
:2066C000A0F707F80F92E8942BE33AEA48EB5FE70E9462320F920F920F924DB75EB70F9289
:2066E0000E945C34E8E6F0E00E94A3334F915F91EF91FF91E595EE1FFF1F49F0FE57E068F7
:206700004427EE0F441FFA95E1F74195550B0E94D6330F9007FE0C94CA3308959F3F31F089
:20672000915020F4879577956795B795880F911D9695879597F9089591505040660F771FBF
:20674000881FD2F70895DF93CF931F930F93FF92EF92DF927B018C01689406C0DA2EEF01BE
:206760000E945F32FE01E894A5912591359145915591A6F3EF010E949330FE019701A801CF
:20678000DA9469F7DF90EF90FF900F911F91CF91DF9108959B01AC0160E070E080E89FE32E
:2067A0000C94ED300C94F6310C948E330E942632D8F39923C9F3940F511DA3F3915050409F
:2067C00094F059F0882332F0660F771F881F91505040C1F79E3F51052CF7880F911D96957E
:2067E000879597F908955F3FACF0983E9CF0BB27869577956795B79508F4B1609395C1F776
:20680000BB0F58F711F460FFE8CF6F5F7F4F8F4F9F4FE3CF0C94413216F00C948E330C9410
:20682000FC3168940C94F6310E942632A8F39923C1F3AEF3DF93CF931F930F93FF92C92F11
:20684000DD2788232AF02197660F771F881FDAF720E030E040E85FEB9FE3883920F0803EA1
:2068600038F021968F770E947C30E0E9F0E004C00E947C30EDEBF0E00E94A3338B01BE01CF
:20688000EC01FB2E6F5771097595771F880B990B0E94973128E132E741E35FE30E945F32A6
:2068A000AF2D9801AE01FF900F911F91CF91DF910E9493300C940D32FA01DC01AA0FBB1F56
:2068C0009B01AC01BF5728F4222733274427507820C0B75190F4AB2F00244695379527959A
:2068E000011CA395D2F3002071F0220F331F441FB395DAF30ED00C947B3061307105A0E84A
:206900008A07B94630F49B01AC016627772788279078309621F02083318342835383089532
:20692000DB018F939F930E943730BF91AF91A29F800D911DA39F900DB29F900D1124089573
:20694000AA1BBB1B51E107C0AA1FBB1FA617B70710F0A61BB70B881F991F5A95A9F78095FF
:206960009095BC01CD01089597FB072E16F4009407D077FD09D00E94A03407FC05D03EF4C1
:20698000909581959F4F0895709561957F4F0895EE0FFF1F0590F491E02D099481E090E01B
:2069A000F8940C94D334F894FFCF010105780682060000050D00000A1A00001A4100003577
:2069C0008200006A0401000A8B020015160500D00700008813000010270000204E00005098
:2069E000C300002C01010100007D9600020200007D4B00050400007D32000A0600007D146D
:206A000000140F00007D0A00321E0000FA0500643C0000FA960000002C010000EE02000030
:206A2000DC050000B80B000000000000500AF304041303133910EB07150DED0C090DFD0CBF
:206A40001C0DEB07A2109C0EB815A515830F8815A10B420B6E616E00696E66006F7666004B
:206A60006D617800617672006D696E00FFFFFFFFFFFFFFFFFFFFFFFFFFFFFFFFFFFFFFFF57
:206A8000BE01EC01FB2E6F5771097595771F880B990B0E94983228E132E741E35FE30E9474
:206AA0006033AF2D9801AE01FF900F911F91CF91DF910E9494310C940E33FA01DC01AA0F97
:206AC000BB1F9B01AC01BF5728F4222733274427507820C0B75190F4AB2F0024469537957A
:206AE0002795011CA395D2F3002071F0220F331F441FB395DAF30ED00C947C316130710512
:206B0000A0E88A07B94630F49B01AC016627772788279078309621F0208331834283538345
:206B20000895DB018F939F930E943831BF91AF91A29F800D911DA39F900DB29F900D11246F
:206B40000895AA1BBB1B51E107C0AA1FBB1FA617B70710F0A61BB70B881F991F5A95A9F775
:206B600080959095BC01CD01089597FB072E16F4009407D077FD09D00E94A13507FC05D0DA
:206B80003EF4909581959F4F0895709561957F4F0895EE0FFF1F0590F491E02D099481E057
:206BA00090E0F8940C94D435F894FFCF010105780682060000050D00000A1A00001A410038
:206BC00000358200006A0401000A8B020015160500D00700008813000010270000204E00B1
:206BE0000050C300002C01010100007D9600020200007D4B00050400007D32000A060000AC
:206C00007D1400140F00007D0A00321E0000FA0500643C0000FA960000002C010000EE029D
:206C20000000DC050000B80B000000000000F209E204D912D812EE0F8D07B70C8F0CAB0C54
:206C40009F0CBE0C8D0767103E0E8D157A152C0F5D15430BE40A6E616E00696E66006F76EF
:206C600066006D617800617672006D696E00FFFFFFFFFFFFFFFFFFFFFFFFFFFFFFFFFFFFED
:206C8000879597F90895E1E0660F771F881FBB1F621773078407BA0720F0621B730B840B85
:206CA000BA0BEE1F88F7E09508950E945C366894B1110C94373708950E941C3788F09F5771
:206CC00098F0B92F9927B751B0F0E1F0660F771F881F991F1AF0BA95C9F714C0B13091F052
:206CE0000E943637B1E008950C943637672F782F8827B85F39F0B93FCCF386957795679544
:206D0000B395D9F73EF490958095709561957F4F8F4F9F4F0895E89409C097FB3EF490958F
:206D20008095709561957F4F8F4F9F4F9923A9F0F92F96E9BB279395F695879577956795F4
:206D4000B795F111F8CFFAF4BB0F11F460FF1BC06F5F7F4F8F4F9F4F16C0882311F096E9BE
:206D600011C0772321F09EE8872F762F05C0662371F096E8862F70E060E02AF09A95660F86
:206D8000771F881FDAF7880F9695879597F90895990F0008550FAA0BE0E8FEEF1616170613
:206DA000E807F907C0F012161306E407F50798F0621B730B840B950B39F40A2661F0232B5E
:206DC000242B252B21F408950A2609F4A140A6958FEF811D811D089597F99F6780E870E074
:206DE00060E008959FEF80EC089500240A941616170618060906089500240A941216130647
:206E0000140605060895092E0394000C11F4882352F0BB0F40F4BF2B11F460FF04C06F5F06
:206E20007F4F8F4F9F4F089557FD9058440F551F59F05F3F71F04795880F97FB991F61F0C2
:206E40009F3F79F087950895121613061406551FF2CF4695F1DF08C0161617061806991F10
:206E6000F1CF86957105610508940895E894BB2766277727CB0197F908950E94C83608F404
:206E80008FEF08950E9455370C9403370E94F53638F00E94FC3620F0952311F00C94EC367B
:206EA0000C94F23611240C9437370E94143770F3959FC1F3950F50E0551F629FF001729F44
:206EC000BB27F00DB11D639FAA27F00DB11DAA1F649F6627B00DA11D661F829F2227B00DE7
:206EE000A11D621F739FB00DA11D621F839FA00D611D221F749F3327A00D611D231F849FBA
:206F0000600D211D822F762F6A2F11249F5750409AF0F1F088234AF0EE0FFF1FBB1F661F52
:206F2000771F881F91505040A9F79E3F510580F00C94EC360C9437375F3FE4F3983ED4F37E
:206F4000869577956795B795F795E7959F5FC1F7FE2B880F911D9695879597F9089519F415
:206F600016F40C94F2360C94FA370E941C37B8F39923C9F3B6F39F57550B87FF0E940838EF
:206F80000024A0E640EA900180585695979528F4805C660F771F881F20F026173707480719
:206FA00030F4621B730B840B202931294A2BA69517940794202531254A2758F7660F771F24
:206FC000881F20F026173707480730F4620B730B840B200D311D411DA09581F7B901842F9F
:206FE0009158880F9695879508950E94C836880B990B08959F3F31F0915020F4879577959D
:207000006795B795880F911D9695879597F9089591505040660F771F881FD2F7089597FB54
:20702000072E16F4009407D077FD09D00E94383807FC05D03EF4909581959F4F0895709572
:2070400061957F4F0895EE0FFF1F0590F491E02D09940E946235332312F48A1B9B0B0C9470
:2070600033380E946235B7FF0895821B930B0895AA1BBB1B51E107C0AA1FBB1FA617B7078F
:2070800010F0A61BB70B881F991F5A95A9F780959095BC01CD01089581E090E0F8940C9420
:2070A0005138F894FFCF0178787841730078787878000200000000630C4F08191618164E7D
:2070C00013FE094C0F240F400F340F530FFE09B713B111D619C31998122A17D80D790D0D53
:2070E0000A006E616E00696E66006F766600FFFFFFFFFFFFFFFFFFFFFFFFFFFFFFFFFFFFD3
:207100000C944C2BEF920F931F93CF93DF93E80134E047FD34E1042E000C550B57FF03C0A2
:20712000519541955109E32E022F242FAE010E94A738CE01DF91CF911F910F91EF90089569
:20714000FB01DC0105900D920020E1F70895A9E0B0E0EDEAF8E30C942C3B6A01F22EB02E52
:20716000102FFBE3AF2EA01608F41BE31F5F012F27E0AE014F5F5F4F0E94063ABC018981FC
:20718000982F9970913009F43FC09BE2E1FC04C09E2D9170E0FC3AC05E2D5071E82FE870E7
:2071A00083FF46C084E0911101C083E0EF2DE81B8F1508F0E0E0D6018E2F20E2552351F152
:2071C000992329F0D6019C93C60101966C0196012D5F3F4FE2FE24C08EE4D6018C9391E4B7
:2071E00011969C93119712968C93D9018E2F90E281111BC0E20FF32FF11D10828EEF9FEF16
:207200002996ECE00C94483B9DE2C6CF90E2C4CF2D9381508111FCCFCE0ED11CE0E0D0CF91
:207220008EE6D6018C9391E6DBCF9D938150E0CF482F447082FF3DC084E0911101C083E040
:207240008F1510F4EF2DE81BD6018E2F20E2552309F1992329F0D6019C93C60101966C01B9
:2072600096012D5F3F4FE2FE1BC089E4D6018C938EE411968C93119786E412968C93D90154
:207280008E2F90E2882309F4B5CF9D938150FACF2D9381508111FCCFCE0ED11CE0E0D9CFAA
:2072A00089E6D6018C938EE611968C93119786E6E4CF9B0177FF02C030E020E0A1E0B0E073
:2072C000911102C0B0E0A0E0F9013196AE0FBF1F8B2C912CBB2009F461C05401EFEFAE1A76
:2072E000BE0AAA0DBB1DFA161B0619F014F04F2D4A1B511188C0E3FC59C07601A42FB0E29A
:20730000A1114FC0C40ED11C992309F45BC040E0D6011196F60190836D01552309F448C086
:20732000012F060F9A81582F507184FF03C0913309F4015010160CF047C0093008F008E00B
:20734000EEE2FE2E5B01A01AB10885019194819491082F3F320729F4D601FC92F601319622
:207360006F016217730794F1021713077CF5DB01A21BB30BAA24A394B12CAC0EBD1EAA0DFC
:20738000BB1D11968C9121503109D601119628153905F4F0F60180836D01DBCFB12CA12C0D
:2073A000A0CFF701B1937F01A150AACF9111B0CFD601942F50E302C05D9391509111FCCF4A
:2073C000C40ED11C40E0ACCF01E0BACF80E3DBCF6217730731F4963388F4953311F455233A
:2073E00069F0F6018083FD01842F90E2811108C0A40FB11D1C9290E080E002CF81E3F1CFC9
:2074000091938150F3CF911183CF8ACF283008F027E03327DA01990F311D87FD91600096DB
:207420006105710539F432602E5F3D9330E32A95E1F708959F3F30F080387105610509F082
:207440003C5F3C5F3D93913008F08068911DDF93CF931F930F93FF92EF92192F987F969513
:20746000E92F96959695E90FFF27EE53FF4F99273327EE24FF24A701E70105900894079446
:2074800028F4360FE71EF81E491F511D660F771F881F991F0694A1F70590079428F4E70EBD
:2074A000F81E491F561FC11D770F881F991F661F0694A1F70590079428F4F80E491F561F30
:2074C000C71FD11D880F991F661F771F0694A1F70590079420F4490F561FC71FD81F990FA6
:2074E000661F771F881F0694A9F784911095177041F0D695C79557954795F794E7941A95DA
:20750000C1F7E8E6F0E068941590159135916591959105907FE27395E118F10A430B560B4B
:20752000C90BD009C0F7E10CF11E431F561FC91FD01D7EF4703311F48A95E6CFE894015084
:2075400030F0080F0AF40027021708F4202F2395022F7A3328F079E37D932A95E9F710C0E2
:207560007D932A9589F6069497956795379517951794E118F10A430B560BC90BD00998F000
:2075800023957E9173957A3308F070E37C932013B8F77E9170617D9330F0839571E37D93A7
:2075A00070E32A95E1F71124EF90FF900F911F91CF91DF91992787FD90950895F999FECF19
:2075C00092BD81BDF89A992780B50895262FF999FECF1FBA92BD81BD20BD0FB6F894FA9A1E
:2075E000F99A0FBE01960895052E97FB1EF400940E940B3B57FD07D00E945D3B07FC03D069
:207600004EF40C940B3B50954095309521953F4F4F4F5F4F089590958095709561957F4F93
:207620008F4F9F4F08950E947F3BA59F900DB49F900DA49F800D911D11240895B7FF0C940E
:20764000133B0E94133B821B930B08952F923F924F925F926F927F928F929F92AF92BF92BA
:20766000CF92DF92EF92FF920F931F93CF93DF93CDB7DEB7CA1BDB0B0FB6F894DEBF0FBE5F
:20768000CDBF09942A88398848885F846E847D848C849B84AA84B984C884DF80EE80FD8078
:2076A0000C811B81AA81B981CE0FD11D0FB6F894DEBF0FBECDBFED010895A1E21A2EAA1B0F
:2076C000BB1BFD010DC0AA1FBB1FEE1FFF1FA217B307E407F50720F0A21BB30BE40BF50B67
:2076E000661F771F881F991F1A9469F760957095809590959B01AC01BD01CF010895A29F19
:20770000B001B39FC001A39F700D811D1124911DB29F700D811D1124911D08955058BB27EF
:20772000AA270E94A63B0C94203D0E94123D38F00E94193D20F039F49F3F19F426F40C9405
:207740000F3D0EF4E095E7FB0C94093DE92F0E94313D58F3BA17620773078407950720F040
:2077600079F4A6F50C94533D0EF4E0950B2EBA2FA02D0B01B90190010C01CA01A001112466
:20778000FF27591B99F0593F50F4503E68F11A16F040A22F232F342F4427585FF3CF46955E
:2077A00037952795A795F0405395C9F77EF41F16BA0B620B730B840BBAF09150A1F0FF0F1D
:2077C000BB1F661F771F881FC2F70EC0BA0F621F731F841F48F4879577956795B795F795CF
:2077E0009E3F08F0B0CF9395880F08F09927EE0F9795879508950E94E53C08F481E008951F
:207800000E94143C0C94203D0E94193D58F00E94123D40F029F45F3F29F00C94093D5111FC
:207820000C94543D0C940F3D0E94313D68F39923B1F3552391F3951B550BBB27AA27621728
:207840007307840738F09F5F5F4F220F331F441FAA1FA9F335D00E2E3AF0E0E832D09150EE
:207860005040E695001CCAF72BD0FE2F29D0660F771F881FBB1F261737074807AB07B0E85F
:2078800009F0BB0B802DBF01FF2793585F4F3AF09E3F510578F00C94093D0C94543D5F3F83
:2078A000E4F3983ED4F3869577956795B795F7959F5FC9F7880F911D9695879597F90895E2
:2078C000E1E0660F771F881FBB1F621773078407BA0720F0621B730B840BBA0BEE1F88F731
:2078E000E09508950E94793C6894B1110C94543D08950E94393D88F09F5798F0B92F9927DD
:20790000B751B0F0E1F0660F771F881F991F1AF0BA95C9F714C0B13091F00E94533DB1E072
:2079200008950C94533D672F782F8827B85F39F0B93FCCF3869577956795B395D9F73EF42A
:2079400090958095709561957F4F8F4F9F4F0895E89409C097FB3EF490958095709561957D
:207960007F4F8F4F9F4F9923A9F0F92F96E9BB279395F695879577956795B795F111F8CFA3
:20798000FAF4BB0F11F460FF1BC06F5F7F4F8F4F9F4F16C0882311F096E911C0772321F00B
:2079A0009EE8872F762F05C0662371F096E8862F70E060E02AF09A95660F771F881FDAF7A8
:2079C000880F9695879597F90895990F0008550FAA0BE0E8FEEF16161706E807F907C0F036
:2079E00012161306E407F50798F0621B730B840B950B39F40A2661F0232B242B252B21F4FD
:207A000008950A2609F4A140A6958FEF811D811D089597F99F6780E870E060E008959FEF70
:207A200080EC089500240A941616170618060906089500240A9412161306140605060895A3
:207A4000092E0394000C11F4882352F0BB0F40F4BF2B11F460FF04C06F5F7F4F8F4F9F4FE2
:207A6000089557FD9058440F551F59F05F3F71F04795880F97FB991F61F09F3F79F08795AD
:207A80000895121613061406551FF2CF4695F1DF08C0161617061806991FF1CF86957105D6
:207AA000610508940895E894BB2766277727CB0197F908950E94E53C08F48FEF08950E9429
:207AC000723D0C94203D0E94123D38F00E94193D20F0952311F00C94093D0C940F3D112419
:207AE0000C94543D0E94313D70F3959FC1F3950F50E0551F629FF001729FBB27F00DB11D02
:207B0000639FAA27F00DB11DAA1F649F6627B00DA11D661F829F2227B00DA11D621F739FF6
:207B2000B00DA11D621F839FA00D611D221F749F3327A00D611D231F849F600D211D822F62
:207B4000762F6A2F11249F5750409AF0F1F088234AF0EE0FFF1FBB1F661F771F881F915044
:207B60005040A9F79E3F510580F00C94093D0C94543D5F3FE4F3983ED4F3869577956795E6
:207B8000B795F795E7959F5FC1F7FE2B880F911D9695879597F9089519F416F40C940F3DF6
:207BA0000C94173E0E94393DB8F39923C9F3B6F39F57550B87FF0E94253E0024A0E640EA37
:207BC000900180585695979528F4805C660F771F881F20F026173707480730F4621B730B82
:207BE000840B202931294A2BA69517940794202531254A2758F7660F771F881F20F0261703
:207C00003707480730F4620B730B840B200D311D411DA09581F7B901842F9158880F96959B
:207C2000879508950E94E53C880B990B08959F3F31F0915020F4879577956795B795880FF9
:207C4000911D9695879597F9089591505040660F771F881FD2F7089597FB072E16F4009414
:207C600007D077FD09D00E94553E07FC05D03EF4909581959F4F0895709561957F4F089575
:207C8000EE0FFF1F0590F491E02D09940E947F3B332312F48A1B9B0B0C94503E0E947F3B78
:207CA000B7FF0895821B930B0895AA1BBB1B51E107C0AA1FBB1FA617B70710F0A61BB70B64
:207CC000881F991F5A95A9F780959095BC01CD01089581E090E0F8940C946E3EF894FFCF51
:207CE00001787878417300787878780002FF835700000000C70F110B0B1A0A1A4416620DA8
:207D0000B0128812A4129812B712620DBD165F14C81DB51D82151C1B3C11DD100D0A006EE5
:207D2000616E00696E66006F76660000FFFFFFFFFFFFFFFFFFFFFFFFFFFFFFFFFFFFFFFF00
:207D4000FFFFFFFFFFFFFFFFFFFFFFFFFFFFFFFFFFFFFFFFFFFFFFFFFFFFFFFFFFFFFFFF43
:207D6000FFFFFFFFFFFFFFFFFFFFFFFFFFFFFFFFFFFFFFFFFFFFFFFFFFFFFFFFFFFFFFFF23
:207D8000FFFFFFFFFFFFFFFFFFFFFFFFFFFFFFFFFFFFFFFFFFFFFFFFFFFFFFFFFFFFFFFF03
:207DA000FFFFFFFFFFFFFFFFFFFFFFFFFFFFFFFFFFFFFFFFFFFFFFFFFFFFFFFFFFFFFFFFE3
:207DC000FFFFFFFFFFFFFFFFFFFFFFFFFFFFFFFFFFFFFFFFFFFFFFFFFFFFFFFFFFFFFFFFC3
:207DE000FFFFFFFFFFFFFFFFFFFFFFFFFFFFFFFFFFFFFFFFFFFFFFFFFFFFFFFFFFFFFFFFA3
:207E0000112484B714BE81FFF0D085E08093810082E08093C00088E18093C10086E08093FC
:207E2000C20080E18093C4008EE0C9D0259A86E020E33CEF91E0309385002093840096BBAD
:207E4000B09BFECF1D9AA8958150A9F7CC24DD2488248394B5E0AB2EA1E19A2EF3E0BF2E79
:207E6000A2D0813461F49FD0082FAFD0023811F0013811F484E001C083E08DD089C0823404
:207E800011F484E103C0853419F485E0A6D080C0853579F488D0E82EFF2485D0082F10E0A0
:207EA000102F00270E291F29000F111F8ED068016FC0863521F484E090D080E0DECF84364D
:207EC00009F040C070D06FD0082F6DD080E0C81680E7D80618F4F601B7BEE895C0E0D1E0ED
:207EE00062D089930C17E1F7F0E0CF16F0E7DF0618F0F601B7BEE89568D007B600FCFDCF1A
:207F0000A601A0E0B1E02C9130E011968C91119790E0982F8827822B932B1296FA010C016F
:207F200087BEE89511244E5F5F4FF1E0A038BF0751F7F601A7BEE89507B600FCFDCF97BE85
:207F4000E89526C08437B1F42ED02DD0F82E2BD03CD0F601EF2C8F010F5F1F4F84911BD0B8
:207F6000EA94F801C1F70894C11CD11CFA94CF0CD11C0EC0853739F428D08EE10CD085E9AE
:207F80000AD08FE07ACF813511F488E018D01DD080E101D065CF982F8091C00085FFFCCF0A
:207FA0009093C60008958091C00087FFFCCF8091C00084FD01C0A8958091C6000895E0E68F
:207FC000F0E098E1908380830895EDDF803219F088E0F5DFFFCF84E1DECF1F93182FE3DF47
:207FE0001150E9F7F2DF1F91089580E0E8DFEE27FF270994FFFFFFFFFFFFFFFFFFFF040425
:00000001FF
